:100000000C9473000C949B000C949B000C949B002C
:100010000C949B000C94E4020C949B000C949B00A9
:100020000C949B000C949B000C949B000C949B00E4
:100030000C949B000C949B000C949B000C949B00D4
:100040000C94D31E0C949B000C94CD170C94A71702
:100050000C949B000C949B000C949B000C949B00B4
:100060000C94FF170C949B00580D5A0D5C0D5E0DFF
:10007000600D620D640D660D970D9A0D9D0D940D2A
:10008000A00DA30DB50DB50D000000002500280042
:100090002B000000000023002600290004040404B3
:1000A0000404040402020202020203030303030322
:1000B00001020408102040800102040810200102FF
:1000C00004081020000000080002010000030407DB
:1000D00000000000000000000000000024002700D5
:1000E0002A00532F0F2F11241FBECFEFD8E0DEBF01
:1000F000CDBF26E0A8E6B4E001C01D92A33DB20743
:10010000E1F714E0A0E0B1E0E0ECFFE602C005900A
:100110000D92A836B107D9F710E0C2E7D0E004C0CD
:100120002197FE010E941E34C137D107C9F70E94F2
:100130001D1F0C94D3370C940000CF93DF93EC0178
:100140008091790490917A04009709F054C08091CD
:100150007C04882309F412C18091770481110EC1B7
:10016000C130D10511F540914F015091500160917E
:100170005101709152018091530190915401A091CD
:100180005501B0915601840F951FA61FB71F811509
:1001900021EE920725EFA20725E0B2070CF408C272
:1001A00080E091EEA5EFB5E003C2CF3F8FEFD80717
:1001B00009F0E4C080914F0190915001A09151014C
:1001C000B0915201409153015091540160915501F9
:1001D00070915601841B950BA60BB70B813AE6E88C
:1001E0009E07E1E0AE07B1050CF0E2C180EA96E8B7
:1001F000A1E0B0E0DDC1019709F05CC06AE471E004
:1002000082E390E00E947619FC0180819181A281B5
:10021000B38180934A0190934B01A0934C01B0931A
:100220004D01C130D10539F5409153015091540130
:100230006091550170915601840F951FA61FB71F3D
:100240008038F3EC9F07F9ECAF07F1E0BF0724F02B
:1002500080E893ECA9ECB1E080934A0190934B01C4
:10026000A0934C01B0934D016AE471E082E390E009
:100270000E94B4191CC0CF3F2FEFD207C1F44091A8
:100280005301509154016091550170915601841BA6
:10029000950BA60BB70B813AE6E89E07E1E0AE07A7
:1002A000B105D4F680EA96E8A1E0B0E0D5CF81E0D0
:1002B00080937B048091790490917A04029709F0ED
:1002C0005DC066E471E08AE090E00E947619FC016E
:1002D00080819181A281B3818093460190934701EF
:1002E000A0934801B0934901C130D10531F5409147
:1002F0005301509154016091550170915601840F42
:10030000951FA61FB71F8034F2E49F07FFE0AF07D9
:10031000B10524F080E492E4AFE0B0E080934601C0
:1003200090934701A0934801B093490166E471E0BE
:100330008AE090E00E94B4191EC0CF3F2FEFD20791
:10034000D1F4409153015091540160915501709145
:100350005601841B950BA60BB70B181619061A0627
:100360001B06E4F2109246011092470110924801D8
:1003700010924901DBCF81E080937B048091790466
:1003800090917A04039709F04AC0C130D10539F53C
:100390008091740690917506A0917606B0917706CB
:1003A000805C944BA34BBF4F8115E9EE9E07E4EAB6
:1003B000AE07E5E3BE0724F080E099EEA4EAB5E3DA
:1003C0008093740690937506A0937606B093770693
:1003D00064E776E08EE190E00E94B4191DC0CF3F43
:1003E000FFEFDF07C9F48091740690917506A09124
:1003F0007606B091770680549B44AC44B1098130B5
:1004000026E4920723ECA20723E2B207CCF680E0B1
:1004100096E4A3ECB3E2D4CF81E080937B04809197
:10042000790490917A04049709F053C0809178047C
:10043000813009F44EC062E471E084E190E00E94F2
:100440007619FC0180819181A281B381C130D105EF
:10045000F9F4805F984DAF4FBF4F8038F3EC9F07A2
:10046000F9ECAF07F1E0BF0724F080E893ECA9ECCA
:10047000B1E08093420190934301A0934401B09373
:10048000450162E471E084E190E00E94B4191EC06D
:10049000CF3F2FEFD20749F0809342019093430161
:1004A000A0934401B093450111C080519742A10926
:1004B000B1098130E6E39E07EEE6AE07E1E0BE0754
:1004C000C4F680E096E3AEE6B1E0D3CF81E080935E
:1004D0007B048091790490917A04059741F568E353
:1004E00071E088E290E00E94E719FC018081C13050
:1004F000D10549F48F5F843008F083E080933801A0
:100500000E94F1190BC0CF3FFFEFDF0719F0809376
:10051000380104C0815091F781E0F0CF81E08093F1
:100520007B0468E371E088E290E00E949C1980916E
:10053000790490917A04069709F043C0C130D1053F
:10054000E9F46EE471E08CE390E00E94E719FC01AD
:100550008081833010F08F5F01C083E080934E0173
:1005600080914E018A3018F08AE080934E016EE44B
:1005700071E08CE390E00E949C1916C02196A1F4D2
:1005800080914E01882381F09EEF980F923010F0F9
:10059000815001C082E080934E0180914E018330F2
:1005A00030F710924E01E3CF81E080937B0409C0C5
:1005B00080934F0190935001A0935101B093520149
:1005C000DDCEDF91CF9108951F920F920FB60F925B
:1005D00011242F933F934F935F936F937F938F9348
:1005E0009F93AF93BF93CF93DF93EF93FF9380914C
:1005F0007B060E940214EC0180917A060E9402148C
:10060000E0917906EF70CC0FDD1F8C2B94E0E99F11
:10061000F0011124EB59FE4FE80FF11D808180930A
:100620007906807339F1803169F481E090E00E94AD
:100630009D008091790490917A04892BD9F467EC1C
:1006400073E00EC08032B1F48FEF9FEF0E949D00E7
:100650008091790490917A04892B61F46BEC73E0BA
:1006600085E695E00E94A51762E370E080E090E0E7
:100670000E948D1EFF91EF91DF91CF91BF91AF91BD
:100680009F918F917F916F915F914F913F912F91AA
:100690000F900FBE0F901F90189580917904909144
:1006A0007A04029799F480913901843078F088EEC9
:1006B00093E0A0E0B0E08093530190935401A093A5
:1006C0005501B093560184E080933901809139013E
:1006D0009091B004891709F449C0813029F481E070
:1006E00090E0A0E0B0E029C0823029F48AE090E0F8
:1006F000A0E0B0E022C0833029F484E690E0A0E0DE
:10070000B0E01BC0843029F488EE93E0A0E0B0E0B4
:1007100014C0853029F480E197E2A0E0B0E00DC07C
:10072000863029F480EA96E8A1E0B0E006C0873080
:1007300069F480E492E4AFE0B0E0809353019093D9
:100740005401A0935501B093560105C0883018F0AC
:1007500087E08093390180913901811103C081E0E4
:1007600080933901809139018093B004089580917C
:100770004E01811102C081E01FC0833011F485E277
:100780001BC0843011F482E317C0853011F481E47A
:1007900013C0863011F48BE40FC0873011F488E564
:1007A0000BC0883011F484E607C0893011F481E76A
:1007B00003C08A3019F48DE7809375046EE471E00C
:1007C0008CE390E00C949C1980914F019091500122
:1007D000A0915101B0915201AC01BD014052514A6A
:1007E0006740710941155F4964427105B8F461E0E1
:1007F0008CE00E942B1460E08BE00E942B1460E0E0
:100800008AE00E942B1460E089E00E942B1460E0D3
:1008100088E00E942B146FEC73E00AC1AC01BD01AB
:10082000405250446C42710940325B406042710555
:10083000B8F460E08CE00E942B1461E08BE00E9431
:100840002B1460E08AE00E942B1460E089E00E9493
:100850002B1460E088E00E942B1463ED73E0E8C085
:10086000AC01BD0140545B446C447109403C564CA2
:100870006D427105B8F460E08CE00E942B1460E0DA
:100880008BE00E942B1461E08AE00E942B1460E050
:1008900089E00E942B1460E088E00E942B1466ED32
:1008A00073E0C6C0AC01BD0152516A4771094115E0
:1008B00059406D437105B8F460E08CE00E942B1440
:1008C00060E08BE00E942B1460E08AE00E942B1411
:1008D00061E089E00E942B1460E088E00E942B1404
:1008E00069ED73E0A5C0AC01BD015B51674B7109B7
:1008F000411559406D437105B8F460E08CE00E94E9
:100900002B1460E08BE00E942B1460E08AE00E94D0
:100910002B1461E089E00E942B1460E088E00E94C3
:100920002B146CED73E084C0AC01BD015452644FD4
:100930007109403C564C6D427105B8F460E08CE0A2
:100940000E942B1460E08BE00E942B1460E08AE090
:100950000E942B1460E089E00E942B1461E088E083
:100960000E942B146FED73E063C0AC01BD01405CCD
:100970005A4E61427140403C564C6D427105B8F48C
:1009800060E08CE00E942B1460E08BE00E942B144E
:1009900060E08AE00E942B1460E089E00E942B1442
:1009A00061E088E00E942B1462EE73E041C0AC016C
:1009B000BD014058514B6F44714040345B446C441E
:1009C0007105B8F460E08CE00E942B1460E08BE0CD
:1009D0000E942B1460E08AE00E942B1460E089E002
:1009E0000E942B1461E088E00E942B1465EE73E0F6
:1009F0001FC0805C9C4FAB49B14080349D45A64CE4
:100A0000B105D0F460E08CE00E942B1460E08BE034
:100A10000E942B1460E08AE00E942B1460E089E0C1
:100A20000E942B1461E088E00E942B1468EE73E0B2
:100A300086E296E00C943A170895CF92DF92EF92F7
:100A4000FF92CF93DF9360E083E00E946C1A609185
:100A50004F0170915001809151019091520120E419
:100A600032E44FE050E00E94FF3369017A012A30FE
:100A7000310518F480E20E94831BC6010E947D1B91
:100A80008EE20E94831B60914F0170915001809112
:100A900051019091520120E432E44FE050E00E9475
:100AA000FF3328EE33E040E050E00E94FF3369015D
:100AB0007A01E9012436310540F480E30E94831B6A
:100AC0002A9718F480E30E94831BC6010E947D1BB5
:100AD0008EE20E94831B60914F01709150018091C2
:100AE00051019091520128EE33E040E050E00E9425
:100AF000FF336B017C01EB016436710540F480E348
:100B00000E94831B2A9718F480E30E94831BC6016E
:100B10000E947D1B6CE273E08AEB96E0DF91CF913F
:100B2000FF90EF90DF90CF900C94A517FF920F935A
:100B30001F93CF93DF93EC01F62E08811981C80132
:100B40000E944E32F81621F06F2DC8010E945632D5
:100B5000CE01DF91CF911F910F91FF9008951F93C8
:100B6000CF93DF93CDB7DEB72C970FB6F894DEBFE7
:100B70000FBECDBF6BEE73E0CE0107960E946D17DE
:100B800060E070E0CE0107960E94C8138823A9F0A8
:100B900065E172E0CE0101960E946D1761E070E0A0
:100BA000CE0101960E94C81311E0811101C010E02E
:100BB000CE0101960E94681701C010E0CE01079691
:100BC0000E9468171123C1F06DED72E085E695E093
:100BD0000E94A51760E080E00E946C1A6DEE73E041
:100BE0008AEB96E00E94A51768EE73E080E090E043
:100BF0000E948D1E0E94B6086EEF73E0CE0107962C
:100C00000E946D1760E070E0CE0107960E94C81345
:100C10008823A9F065E172E0CE0101960E946D176C
:100C200061E070E0CE0101960E94C81311E08111CD
:100C300001C010E0CE0101960E94681701C010E0CB
:100C4000CE0107960E946817112329F081E0809356
:100C50007D040E94B60860E074E0CE0107960E9411
:100C60006D1760E070E0CE0107960E94C8138823DC
:100C7000A9F065E172E0CE0101960E946D1765E270
:100C800070E0CE0101960E94C81311E0811101C0ED
:100C900010E0CE0101960E94681701C010E0CE015D
:100CA00007960E946817112309F44CC14DE050E0EB
:100CB00062E070E0CE0101960E94A81DBE016F5F48
:100CC0007F4F88E696E00E94BA16CE0101960E94F8
:100CD000681788E696E00E94811660934F01709332
:100CE000500180935101909352018091780481309A
:100CF000A1F480917604813081F48091AC049091CC
:100D0000AD04A091AE04B091AF0480934F019093D5
:100D10005001A0935101B093520180917B04811145
:100D200010C080917C0481110CC080917904909155
:100D30007A04892B31F481E10E940214019709F4AD
:100D400008C24EE150E06DE170E0CE0101960E94D4
:100D5000A81DBE016F5F7F4F80E596E00E94BA1626
:100D6000CE0101960E94681780E596E00E948116E8
:100D7000613029F410926F0463E074E039C062308E
:100D800029F460936F0466E074E032C0633031F49C
:100D900084E080936F0469E074E02AC0643031F429
:100DA00085E080936F046CE074E022C0653031F41C
:100DB00086E080936F046FE074E01AC0663031F40F
:100DC00089E080936F0462E174E012C0673031F40F
:100DD00083E080936F0465E174E00AC0693019F024
:100DE00060936F0409C087E080936F0468E174E04A
:100DF00080E596E00E943A1741E250E060E270E040
:100E0000CE0101960E94A81DBE016F5F7F4F82E355
:100E100096E00E94BA16CE0101960E94681782E3FE
:100E200096E00E9481166093760448E150E067E105
:100E300070E0CE0101960E94A81DBE016F5F7F4F3A
:100E40008CE596E00E94BA16CE0101960E946817C2
:100E50008CE596E00E94811660936E0449E150E0B3
:100E600068E170E0CE0101960E94A81DBE016F5F8F
:100E70007F4F86E596E00E94BA16CE0101960E9449
:100E8000681786E596E00E94811660936D0442E142
:100E900050E061E170E0CE0101960E94A81DBE0104
:100EA0006F5F7F4F88E396E00E94BA16CE010196ED
:100EB0000E94681747E150E062E170E0CE010196C0
:100EC0000E94A81DBE016F5F7F4F84E496E00E94E0
:100ED000BA16CE0101960E94681784E496E00E943B
:100EE00081166093690470936A0480936B049093F5
:100EF0006C044DE150E06CE170E0CE0101960E947F
:100F0000A81DBE016F5F7F4F82E696E00E94BA1671
:100F1000CE0101960E94681782E696E00E94811633
:100F200060937804613039F480917C04811103C0AE
:100F30006093730402C0109273041092680481E0FD
:100F400080937D046BE174E0CE0107960E946D17DB
:100F500060E070E0CE0107960E94C8138823A9F0D4
:100F600065E172E0CE0101960E946D1768E070E0C5
:100F7000CE0101960E94C81311E0811101C010E05A
:100F8000CE0101960E94681701C010E0CE010796BD
:100F90000E9468171123E9F048E050E065E070E036
:100FA000CE0101960E94A81DBE016F5F7F4F8EE3A8
:100FB00096E00E94BA16CE0101960E9468178EE351
:100FC00096E00E94811670937104609370041092F1
:100FD000680461E274E0CE0107960E946D1760E03C
:100FE00070E0CE0107960E94C8138823A9F065E13E
:100FF00072E0CE0101960E946D1765E070E0CE01AF
:1010000001960E94C81311E0811101C010E0CE01C9
:1010100001960E94681701C010E0CE0107960E9459
:101020006817112309F449C045E050E064E070E01E
:10103000CE0101960E94A81DBE016F5F7F4F80E226
:1010400096E00E94BA16CE0101960E94681780E2CF
:1010500096E00E94811660937204611108C061E0FD
:1010600087E00E942B1460E086E00E942B148091A0
:101070007204813041F460E087E00E942B1460E04C
:1010800086E00E942B1480917204823041F461E06A
:1010900087E00E942B1461E086E00E942B1480916F
:1010A0007204833041F460E087E00E942B1461E019
:1010B00086E00E942B141092680466E274E0CE0170
:1010C00007960E946D1760E070E0CE0107960E94BF
:1010D000C8138823A9F065E172E0CE0101960E9451
:1010E0006D176DE070E0CE0101960E94C81311E00B
:1010F000811101C010E0CE0101960E94681701C065
:1011000010E0CE0107960E946817112329F14DE0E7
:1011100050E063E070E0CE0101960E94A81DBE0180
:101120006F5F7F4F8AE196E00E94BA16CE0101966A
:101130000E9468178AE196E00E9481166093AC04D1
:101140007093AD048093AE049093AF041092680442
:1011500003C00E941D05F5CD2C960FB6F894DEBF96
:101160000FBECDBFDF91CF911F91089585E695E029
:101170000E946D1569E274E085E695E00E94A5176E
:101180006091740470E080E090E00E948D1E85E61E
:1011900095E00E94E814892B09F068C08091AA04A8
:1011A0009091AB0401969093AB048093AA04883C81
:1011B00091050CF45BC08091790490917A04892B9D
:1011C00009F054C080917C04811150C08091A90421
:1011D0008F5F8093A904823070F460E080E00E9409
:1011E0006C1A6DE274E08AEB96E00E94A51761E04C
:1011F0008DE00E942B148091A9048250823080F4EB
:1012000060E080E00E946C1A6EE374E08AEB96E086
:101210000E94A51760E08DE00E942B141092A90493
:1012200061E080E00E946C1A60E574E08AEB96E071
:101230000E94A51780E20E94831B60913E0170917D
:101240003F0180914001909141010E94741265E537
:1012500074E08AEB96E00E94A51780E20E94831B4F
:101260001092AB041092AA041092770485E695E0E0
:101270000E94E81418161906ECF466E372E08EE694
:1012800096E00E943A1785E695E00E94E814181649
:1012900019066CF485E695E00E94C6140E94ED13D1
:1012A00061E070E080E090E00E948D1EECCF81E074
:1012B0008093680480916804882369F00E94AF05D8
:1012C0001092AB041092AA0481E08093770461E04D
:1012D0008DE00C942B1408952F923F924F925F92C1
:1012E0006F927F928F929F92AF92BF92CF92DF9236
:1012F000EF92FF920F931F93CF93DF93CDB7DEB79B
:1013000068970FB6F894DEBF0FBECDBF522E3D8753
:10131000442E5E873B011C01A982B98ACA8ADB8AF6
:10132000EC8AFD8A0E8B1F8B988A8F86211500EA26
:1013300030070CEA400709EB500703E0600771052E
:101340008105910511F008F046C02F3F10EE3107DE
:1013500015EF410715E051076105710581059105FC
:1013600061F058F02F3F354D41415E4763407105B4
:101370008105910509F0D8F50BC0512CF1EEFD87E0
:10138000B5EF4B2E05E00E87612C712C212C312CF2
:10139000298139894A895B896C897D898E899F89F0
:1013A000A0E00E94A03509F0A7C0A52CBD84C42CE4
:1013B000DE847301810120E034E04BE654EF64E108
:1013C00070E080E090E00E94EA3429873A874B87FA
:1013D0005C87912C24C0512C10EA1D87FCEA4F2E0B
:1013E00029EB2E87A3E06A2E712C212C312C298128
:1013F00039894A895B896C897D898E899F89A0E0BA
:101400000E94A03509F0F4C09924939414E0E12ED1
:10141000F12C00E010E0E986FA860B871C87E9844E
:10142000FA840B851C85A801970160E070E0CB0170
:10143000A52CBD84C42CDE847301810129833A83E9
:101440004B835C836D837E838F83988760E070E03D
:1014500080E090E00E9424342983398B4A8B5B8B97
:101460006C8B7D8B8E8B9F8BFF24F3949F1409F4E0
:10147000C2C010E0812C912C5401839440E050E0D4
:10148000BA0101C011E0CB01BA0107E0660F771F76
:10149000881F991F0A95D1F7C984DA84EB84FC84EC
:1014A00027E0CC0CDD1CEE1CFF1C2A95D1F7A2E036
:1014B000DA1AE108F108A50194010E94DD33C20E99
:1014C000D31EE41EF51EEF85F889C082D182E28228
:1014D000F382648375838683978380869186A28650
:1014E000B3861111BBC0298139894A895B896C890E
:1014F0007D898E899F89B8C0188EA52CBD84C42C87
:10150000DE8473018101298139894A895B896C896B
:101510007D898E899F890E94EA3429873A874B8783
:101520005C8789859A85AB85BC850697A105B10541
:1015300020F4B6E0AB2EB12C0FC0E984FA840B8501
:101540001C8529E0E21627E0F20601051105D0F01E
:10155000F8E0AF2EA7E0BA2EC12CD12CE12CF12C53
:1015600000E010E0298139894A895B896C897D898D
:101570008E899F890E94EA34522E3D87442E5E87D1
:101580003B011C01A52CBD84C42CDE8473018101A8
:10159000298139894A895B896C897D898E899F89EE
:1015A0000E94E834AA24AA94BB24BA94EFE0CE2E79
:1015B000D12CE12CF12C00E010E00E942434A52C69
:1015C000BD84C42CDE84730181010E94EA34A32F00
:1015D000F42FE52F422F5A2F6F2F7E2F41155105E3
:1015E00061057105F9F4812C912C5401839420C07C
:1015F00081E0888F82CFAF85B8891D921D921D92A0
:101600001C921397FD011482158216821782C12C39
:10161000D12C7601C3941896CD92DD92ED92FC9276
:101620001B9722C088248A94982C8FE0A82EB12C76
:10163000F88DF13009F026CFEF85F88910821182FC
:1016400012821382148215821682178281E090E042
:10165000A0E0B0E080879187A287B387252D3D85E4
:10166000442D5E85B301C10168960FB6F894DEBFC4
:101670000FBECDBFDF91CF911F910F91FF90EF90E3
:10168000DF90CF90BF90AF909F908F907F906F90A2
:101690005F904F903F902F900895DF92EF92FF92CE
:1016A0000F931F93CF93DF93FC01E080F1800281C1
:1016B0001381D481C581B681D7809701A8016D2F90
:1016C0007C2F8B2F9D2D35534C4051096109710999
:1016D000810991092F3F34434C4051056105710543
:1016E0008105910509F098F49701A8016D2F7C2FD1
:1016F0008B2F9D2D07E00E94573520833183428335
:101700005383648375838683978387E0FDC0970145
:10171000A8016D2F7C2F8B2F9D2D3A5648415109E2
:1017200061097109810991092F3F394648415105E5
:10173000610571058105910509F098F49701A801EB
:101740006D2F7C2F8B2F9D2D06E00E945735208317
:10175000318342835383648375838683978386E0D2
:10176000D3C09701A8016D2F7C2F8B2F9D2D345D49
:101770004043510961097109810991092F3F334D96
:1017800040435105610571058105910509F098F403
:101790009701A8016D2F7C2F8B2F9D2D05E00E94B6
:1017A00057352083318342835383648375838683D3
:1017B000978385E0A9C09701A8016D2F7C2F8B2FFF
:1017C0009D2D385A414651096109710981099109D4
:1017D0002F3F374A41465105610571058105910545
:1017E00009F098F49701A8016D2F7C2F8B2F9D2D68
:1017F00004E00E94573520833183428353836483FE
:1018000075838683978384E07FC09701A8016D2F3D
:101810007C2F8B2F9D2D3055434C51096109710947
:10182000810991092F3F3F44434C510561057105E2
:101830008105910509F098F49701A8016D2F7C2F7F
:101840008B2F9D2D03E00E945735208331834283E7
:101850005383648375838683978383E055C09701A0
:10186000A8016D2F7C2F8B2F9D2D305A464851405B
:1018700061097109810991092F3F3F49464851404B
:10188000610571058105910509F098F49701A8019A
:101890006D2F7C2F8B2F9D2D02E00E9457352083CA
:1018A000318342835383648375838683978382E085
:1018B0002BC09701A8016D2F7C2F8B2F9D2D3054AD
:1018C0004D40534061097109810991092F3F3F4300
:1018D0004D405340610571058105910509F098F46B
:1018E0009701A8016D2F7C2F8B2F9D2D01E00E9469
:1018F0005735208331834283538364837583868382
:10190000978381E001C080E0DF91CF911F910F911B
:10191000FF90EF90DF900895CF93DF9391E0909345
:10192000410590E69093630510924205109264057C
:10193000682F82E096E00E9426160E94101A80917D
:1019400040058111FCCF81E08093400510923F0556
:101950009FEF90933E0510923D0510923C058093B9
:101960001B0580911B05806C80931B0580911A05D7
:10197000813061F410921A0580911B058093BB00A1
:101980008091BC0083FDF8CF85EC01C085EE80938B
:10199000BC00809140058130E1F380913D058111CB
:1019A00003C0C0913D0501C0C1E0ECE1F5E0A7EB4B
:1019B000B4E080E08C1721F091919D938F5FFACF76
:1019C0001092B604C093B5048091B604C81731F0E4
:1019D00082E096E00E94DD15D82FF6CF8D2FDF91A3
:1019E000CF9108952F923F924F925F926F927F9284
:1019F0008F929F92AF92BF92CF92DF92EF92FF921F
:101A00000F931F93CF93DF93CDB7DEB72E970FB60B
:101A1000F894DEBF0FBECDBF3C01C982DA82EB82F3
:101A2000FC820D831E832F83388749875A876B87F3
:101A30007C878BA18D873C2C2D2C5E2C0E87412E14
:101A4000922EC984DA84EB84FC8484E190E00E94C5
:101A5000C0358C01FC01D082C182862D880F880F91
:101A6000880F845D0E948C0C952D93708C7F892B40
:101A7000F801828323823482D701C6017CE0B695C7
:101A8000A795979587957A95D1F7807F992D9F7027
:101A9000C92EC80EC58246828E85878398E0691656
:101AA0007104B8F4F301EC5CFF4FB8010C941E34E0
:101AB0008AE20DC082E30BC08AE309C082E407C05A
:101AC0008AE405C082E503C08AE501C08BE50E9477
:101AD000CB1B60E1F62EF60C8F2D0E948C0CE1E002
:101AE000682FAE1202C0606401C06F7B8F2D0E9410
:101AF0008F1DF1E06F16710459F038F092E069160D
:101B0000710449F4A092AF0618C0A092AD060FC0B0
:101B1000A092AE060FC0E8E06E167104B0F4F301B7
:101B2000E45CFF4F0C941E3454E4B52E0EC04CE21E
:101B3000B42E0BC034E3B32E08C02CE3B22E05C084
:101B40009CE4B92E02C084E5B82E8B2D0E948C0C2B
:101B50008378FD85F1118C6090E1899E400111240C
:101B6000682F68298B2D0E948F1DC8012E960FB6F5
:101B7000F894DEBF0FBECDBFDF91CF911F910F91C3
:101B8000FF90EF90DF90CF90BF90AF909F908F909D
:101B90007F906F905F904F903F902F900C945836AD
:101BA0000F931F93CF938B01C0E1C80F8C2F0E941E
:101BB0008C0C0115110511F48F7D04C00130110545
:101BC00009F48062682F8C2FCF911F910F910C9494
:101BD0008F1D2F923F924F925F926F927F928F92C2
:101BE0009F92AF92BF92CF92DF92EF92FF920F93AC
:101BF0001F93CF93DF93CDB7DEB7AB970FB6F894B3
:101C0000DEBF0FBECDBF298F3A8F4B8F5C8F6D8F9C
:101C10007E8F8F8F98A37A2CB9A2CAA2DBA23E2C0A
:101C20004F2C602E212E9AA689A62A2D3B2DA60187
:101C30006E2D7F2D802F912FA0E00E94A03591F076
:101C400038554744584F6D40710981099109211554
:101C50003C4A43425C4F664071058105910511F095
:101C600008F024C4298D3A8D4B8D5C8D6D8D7E8D51
:101C70008F8D98A12F3F34434C405105610571056C
:101C80008105910509F050F4198E85E38A8F8CE067
:101C90008B8F1C8E1D8E1E8E1F8E18A2298D3A8D45
:101CA0004B8D5C8D6D8D7E8D8F8D98A12115304A69
:101CB0004C4A594B634071058105910569F060F00C
:101CC000198E80EA8A8F8CEA8B8F89EB8C8F83E068
:101CD0008D8F1E8E1F8E18A2CE0149960E944D0B2D
:101CE0008BA7272D39A14AA15BA1632D742D862DC9
:101CF000922DA0E0B98DFA8DEB8D0E94A03509F4EC
:101D000081C0AC8D8D8D5E8C9F8D9EA318A118A770
:101D10002B2F3F2F4E2F5A2F682F752D892F912F44
:101D20002F3F15ED310711E141071EE7510713E081
:101D3000610771058105910511F008F063C0CE01BE
:101D40000D964C01A72CB9A0CAA0DBA0E32CF42C63
:101D5000062D122D8EA198A50E946C0989A59AA521
:101D600081309105B1F1E0F0029709F078C3898DD7
:101D70008093A5068A8D8093A6068B8D8093A706F7
:101D80008C8D8093A8068D8D8093A9068E8D80936F
:101D9000AA068F8D8093AB0688A18093AC065FC3A3
:101DA000898D809395068A8D809396068B8D80937E
:101DB00097068C8D809398068D8D809399068E8DD5
:101DC00080939A068F8D80939B0688A180939C06B2
:101DD00046C3898D80939D068A8D80939E068B8D48
:101DE00080939F068C8D8093A0068D8D8093A10695
:101DF0008E8D8093A2068F8D8093A30688A18093F9
:101E0000A4062DC39C8D1D8D1CA35E8C8F8D8EA36F
:101E1000A8A12B2F3F2F4E2F592F612F752D9A2FB1
:101E20002F3F15ED310711E141071EE7510713E080
:101E30006107710581059105D9F0D0F0CE010D96AD
:101E40004C01A12CB12CC12CD12CE12CF12C00E0A7
:101E500010E08EA19A2F0E946C09722E39A34AA31A
:101E60005BA3362E472E682E292E91E09FA301C03A
:101E70001FA289A59AA58130910509F458C020F0C8
:101E8000029709F49EC112C3298D3A8D4B8D5C8D4A
:101E90006D8D7E8DCE010D964C01A12CB12CC12CE7
:101EA000D12CE12CF12C00E010E08F8D98A10E9444
:101EB0006C09722E39A34AA35BA3362E472E682ED7
:101EC000292E60E070E080E090E00E94D00D7092DA
:101ED000850699A190938606EAA1E09387061BA147
:101EE000109388063092890640928A0660928B068B
:101EF00020928C06898D809395068A8D8093960614
:101F00008B8D809397068C8D809398068D8D809312
:101F100099068E8D80939A068F8D80939B0688A15B
:101F200080939C06552453941DA21CA29AC28091B2
:101F3000B506E98DECA3EA8DEEA3EB8DE8A75C8CEA
:101F4000BD8DAE8DFF8DE8A1823009F075C02CA14A
:101F50003EA148A5552D6B2F7A2F8F2F9E2F3058DD
:101F60004A41564061097109810991092F37304E64
:101F700042475849624071058105910569F160F158
:101F8000A090A506B090A606C090A706D090A8067F
:101F9000E090A906F090AA060091AB061091AC065D
:101FA0002CA13EA148A5552D6B2F7A2F8F2F9E2F48
:101FB0000E94973589F010929D0610929E0610920D
:101FC0009F061092A0061092A1061092A2061092EF
:101FD000A3061092A4066AC270908D0680918E06A8
:101FE00089A390918F069AA3109190061BA330901D
:101FF0009106409092066090930620909406CE0140
:102000000D964C01A72CB9A0CAA0D12EE32CF42C1C
:10201000062D122D2CA13EA148A5552D6B2F7A2FF0
:102020008F2F9E2F0E946C0961E070E081E090E0AC
:102030000E94D00D512C38C070928D0699A19093BA
:102040008E061AA110938F068BA180939006309272
:102050009106409292066092930620929406CE01D9
:102060000D964C01A12CB12CC12CD12CE12CF12CC2
:1020700000E010E02CA13EA148A5552D6B2F7A2F32
:102080008F2F9E2F0E946C09722E39A34AA35BA347
:10209000362E472E682E292E61E070E081E090E018
:1020A0000E94D00D55245394298D3A8D4B8D5C8D13
:1020B0006D8D7E8D8F8D98A130584A4156406109B3
:1020C0007109810991092F37304E424758496240C2
:1020D00071058105910509F008F457C081E08093EE
:1020E000B5062091A5063091A6064091A70650910D
:1020F000A8066091A9067091AA068091AB069091FE
:10210000AC06A0E00E94A03509F442C085EA96E042
:102110000E944D0B8BA7A0908D06B0908E06C090AC
:102120008F06D0909006E0909106F0909206009174
:102130009306109194062091A5063091A606409131
:10214000A7065091A8066091A9067091AA06CE0133
:1021500001964C018091AB069091AC060E946C09EF
:102160001F928BA4A12CC980DA80EB80FC800D81AA
:102170001E812F81388549855A856B857C8582E053
:1021800090E00E94F20C0F9003C088E08093B506A7
:10219000898D80939D068A8D80939E068B8D80937A
:1021A0009F068C8D8093A0068D8D8093A1068E8DC9
:1021B0008093A2068F8D8093A30688A18093A406A6
:1021C00049C19090B506E98DECA3EA8DEEA3EB8DA5
:1021D000E8A75C8CBD8DAE8DFF8DE8A111E091125A
:1021E00075C02CA13EA148A5552D6B2F7A2F8F2F9E
:1021F0009E2F30584A415640610971098109910961
:102200002F37304E4247584962407105810591058C
:1022100069F160F1A090A506B090A606C090A7064F
:10222000D090A806E090A906F090AA060091AB060F
:102230001091AC062CA13EA148A5552D6B2F7A2FED
:102240008F2F9E2F0E94973589F01092A50610922D
:10225000A6061092A7061092A8061092A906109240
:10226000AA061092AB061092AC0624C170908D069F
:1022700080918E0689A390918F069AA31091900663
:102280001BA3309091064090920660909306209098
:102290009406CE010D964C01A72CB9A0CAA0D12E50
:1022A000E32CF42C062D122D2CA13EA148A5552D72
:1022B0006B2F7A2F8F2F9E2F0E946C0961E070E0A8
:1022C00082E090E00E94D00D512C38C070928D06B3
:1022D00099A190938E061AA110938F068BA18093DB
:1022E0009006309291064092920660929306209258
:1022F0009406CE010D964C01A12CB12CC12CD12CF1
:10230000E12CF12C00E010E02CA13EA148A5552DB8
:102310006B2F7A2F8F2F9E2F0E946C09722E39A35C
:102320004AA35BA3362E472E682E292E61E070E06B
:1023300082E090E00E94D00D55245394298D3A8D6F
:102340004B8D5C8D6D8D7E8D8F8D98A130584A415F
:10235000564061097109810991092F37304E424772
:102360005849624071058105910509F008F457C08C
:1023700082E08093B50620919D0630919E064091A3
:102380009F065091A0066091A1067091A2068091CF
:10239000A3069091A406A0E00E94A03509F442C0D3
:1023A0008DE996E00E944D0B8BA7A0908D06B09012
:1023B0008E06C0908F06D0909006E0909106F09027
:1023C0009206009193061091940620919D063091FB
:1023D0009E0640919F065091A0066091A1067091C3
:1023E000A206CE0101964C018091A3069091A4060D
:1023F0000E946C091F928BA4A12CC980DA80EB800B
:10240000FC800D811E812F81388549855A856B8519
:102410007C8581E090E00E94F20C0F9003C088E080
:102420008093B506898D8093A5068A8D8093A60634
:102430008B8D8093A7068C8D8093A8068D8D8093BD
:10244000A9068E8D8093AA068F8D8093AB0688A1F6
:102450008093AC0681E090E09DA38CA302C01FA2F4
:10246000512C9FA19F938BA4AFA0CD84DE84EF84D9
:10247000F88809891A892B893C894D895E896F8979
:10248000788D89A59AA50E94F20C0F90E1E05E126A
:1024900010C00CA11DA1272D39A14AA15BA1632D5C
:1024A000742D862D922D0E94F01B03C099249394C5
:1024B00001C0912C892DAB960FB6F894DEBF0FBEEC
:1024C000CDBFDF91CF911F910F91FF90EF90DF90E3
:1024D000CF90BF90AF909F908F907F906F905F90C4
:1024E0004F903F902F900895CF92DF92EF92FF92FE
:1024F000CF93DF9397FF19C06B017C018DE20E949F
:10250000831BEC0166277727CB016C197D098E09A7
:102510009F094AE00E943A1B8C0F9D1FDF91CF91CB
:10252000FF90EF90DF90CF9008954AE0DF91CF9138
:10253000FF90EF90DF90CF900C943A1B009769F0DA
:10254000FC0101900020E9F73197AF01481B590BBE
:10255000BC0184E196E00C948C1680E00895FC01A7
:1025600080913C0690913D06892B21F421E0309723
:1025700049F413C08091380690913906309731F4B0
:1025800021E0FC018081882341F006C0BF010E9448
:10259000B53721E0892B09F020E0822F08958F9232
:1025A0009F92AF92BF92CF92DF92EF92FF920F93E2
:1025B0001F93CF93DF936B017C01142F9B01AC0120
:1025C0000E94C433882319F06BE574E027C04601EC
:1025D0005701E894B7F82FEF3FEF4FE75FE7C501EA
:1025E000B4010E94C43381110DC02FEF3FEF4FE7BC
:1025F0005FE7C501B4010E942A3118161CF46FE58B
:1026000074E00CC02FEF3FEF4FE75FE4C701B60166
:102610000E94BF33181694F463E674E08AEB96E0E8
:10262000DF91CF911F910F91FF90EF90DF90CF90AE
:10263000BF90AF909F908F900C9490172FEF3FEF2B
:102640004FE75FECC701B6010E942A3187FDE4CF56
:1026500020E030E0A901C701B6010E942A3187FFBE
:1026600009C08DE20E94831BEC01F7FAF094F7F8A1
:10267000F09402C0C0E0D0E000E060E070E080E0F4
:102680009FE3101741F020E030E040E251E40E9467
:1026900017330F5FF6CFA70196010E94AB326B0193
:1026A0007C010E9490334B015C014AE00E943A1B7E
:1026B000C80FD91F112399F1C501B4010E942F3110
:1026C0009B01AC01C701B6010E94AA326B017C01DB
:1026D0008EE20E94831BC80FD91F20E030E040E249
:1026E00051E4C701B6010E9490314B015C010E9488
:1026F00090336B017C01CB010E947D1BC80FD91F59
:10270000B60180E090E00E942F319B01AC01C50131
:10271000B4010E94AA326B017C011150F1F6CE0186
:10272000DF91CF911F910F91FF90EF90DF90CF90AD
:10273000BF90AF909F908F90089540E061E08AEB4A
:1027400096E00E9459198BE39FE10197F1F70895F4
:102750000F931F93CF93DF938B01877098E0899F2E
:10276000B0011124606440E08AEB96E00E945919A0
:10277000E801085F1F4F69918AEB96E00E9470198B
:10278000C017D107C1F7DF91CF911F910F91089525
:10279000DC0114964D915C91159720917206309151
:1027A0007306241B350B26173707A0F020916E0601
:1027B00030916F062115310569F0ED91FC9130974C
:1027C00049F0CB01BF01820F931F0E94C53721E062
:1027D000892B09F020E0822F0895CF93DF9300D05A
:1027E000CDB7DEB789831A8241E050E0BE016F5F4A
:1027F0007F4F8EE696E00E948C160F900F90DF912F
:10280000CF910895CF93DF93282F30E0F901EC5357
:10281000FF4F8491F901E055FF4FD491F901E4563F
:10282000FF4FC491CC2391F081110E94111EEC2F17
:10283000F0E0EE0FFF1FEE56FF4FA591B491EC9123
:10284000ED2381E090E021F480E002C080E090E0A0
:10285000DF91CF9108951F93CF93DF93282F30E01E
:10286000F901EC53FF4F8491F901E055FF4FD491EA
:10287000F901E456FF4FC491CC23C1F0162F81110A
:102880000E94111EEC2FF0E0EE0FFF1FE857FF4FE4
:10289000A591B4919FB7F894111104C08C91D09573
:1028A000D82302C0EC91DE2BDC939FBFDF91CF9148
:1028B0001F9108951092B6041092B504109242052B
:1028C000109264051092400581E080933F051092BC
:1028D0001A0561E082E10E942B1461E083E10E940D
:1028E0002B14E9EBF0E080818E7F808380818D7FE7
:1028F000808388E48093B80085E48093BC008BECEF
:1029000095E19093B4048093B3048CEC95E190939B
:10291000B2048093B10408950895CF92DF92EF92AC
:10292000FF920F931F93CF93DF936C017A018B017A
:10293000C0E0D0E0CE15DF0581F0D8016D918D01AA
:10294000D601ED91FC910190F081E02DC601099531
:10295000892B11F02196EECF7E01C701DF91CF9137
:102960001F910F91FF90EF90DF90CF900895FC01A1
:10297000538D448D252F30E0842F90E0821B930BE4
:10298000541710F0CF96089501970895FC01918D8A
:10299000828D981761F0828DDF01A80FB11D5D96C1
:1029A0008C91928D9F5F9F73928F90E008958FEF2F
:1029B0009FEF0895FC01918D828D981731F0828DE3
:1029C000E80FF11D858D90E008958FEF9FEF08953A
:1029D000FC01918D228D892F90E0805C9F4F821B9E
:1029E00091098F739927089585E695E00E94E81470
:1029F00021E0892B09F420E0822F0895FC01848DC9
:102A0000DF01A80FB11DA35ABF4F2C91848D90E018
:102A100001968F739927848FA689B7892C93A089F3
:102A2000B1898C91837080648C93938D848D98137D
:102A300006C00288F389E02D80818F7D8083089510
:102A4000EF92FF920F931F93CF93DF93EC0181E0FE
:102A5000888F9B8D8C8D981305C0E889F9898081BA
:102A600085FD26C0F62E0B8D10E00F5F1F4F0F73F4
:102A70001127E02E8C8DE8120CC00FB607FCFACFA0
:102A8000E889F989808185FFF5CFCE010E94FE1487
:102A9000F1CF8B8DFE01E80FF11DE35AFF4FF0825D
:102AA0009FB7F8940B8FEA89FB89808180620AC006
:102AB0009FB7F894EE89FF896083E889F98980815E
:102AC0008370806480839FBF81E090E0DF91CF912D
:102AD0001F910F91FF90EF900895CF93DF93EC013A
:102AE000888D8823C9F0EA89FB89808185FD05C02E
:102AF000A889B9898C9186FD0FC00FB607FCF5CF68
:102B0000808185FFF2CFA889B9898C9185FFEDCFAF
:102B1000CE010E94FE14E7CFDF91CF91089580E0AF
:102B200090E0892B29F00E94F41481110C9400008C
:102B3000089585ED8093BC008091BC0084FDFCCF9E
:102B40001092400508954091F704262F30E0240F9D
:102B5000311D21323105DCF4209140052430C9F4C7
:102B6000FC0180E090E0861758F43091F704219141
:102B7000DC01A952BB4FA30FB11D2C930196F3CFDB
:102B80008091F704680F6093F70480E0089581E076
:102B9000089582E00895089508950895E091B60497
:102BA0008091B504E81730F4F0E0E954FB4F8081E0
:102BB00090E008958FEF9FEF08959091B604809173
:102BC000B504981750F4E92FF0E0E954FB4F208149
:102BD00030E09F5F9093B60402C02FEF3FEFC90132
:102BE00008958091B50490E02091B604821B91096C
:102BF0000895CF92DF92EF92FF920F931F93CF939E
:102C0000DF937C01CB018A0120914105222389F0C9
:102C1000EB016B01C40ED51ECC15DD0569F0699181
:102C2000D701ED91FC910190F081E02DC70109954C
:102C3000F3CF642F0E94A315C801DF91CF911F919C
:102C40000F91FF90EF90DF90CF900895CF93DF9397
:102C50001F92CDB7DEB76983209141052223D1F0C1
:102C600020916405203240F021E030E0FC01338304
:102C7000228380E090E015C080914205E82FF0E0CB
:102C8000ED5BFA4F998190838F5F8093420580932B
:102C9000640505C061E0CE0101960E94A31581E0A4
:102CA00090E00F90DF91CF91089580E090E008953B
:102CB0000E94A7370F931F93CF93DF93EC01888176
:102CC0009981009729F02A813B812617370788F4DC
:102CD0008B016F5F7F4F0E94E136009761F099830F
:102CE00088831B830A832C813D81232B11F4FC01F3
:102CF000108281E001C080E0DF91CF911F910F91A0
:102D00000895FC0180819181009711F00C94883026
:102D100060E070E0CB010895EF92FF920F931F9354
:102D2000CF93DF936115710511F480E01CC041154C
:102D30005105C1F07B01EC018C819D818A01080F56
:102D4000191FB801CE010E945A16882371F32881F9
:102D500039818C819D81B701820F931F0E94BE37FC
:102D60001D830C8381E0DF91CF911F910F91FF9024
:102D7000EF9008950F931F93CF93DF938C01EB0196
:102D8000FC0180819181009739F06881798161151A
:102D90007105A1F40E94583688819981F8019183C8
:102DA00080838A819B81938382838C819D8195839B
:102DB0008483198218821B821A820FC0F801428113
:102DC00053812C813D814217530720F30E94BE3767
:102DD0008C819D81F801958384831D821C82DF9103
:102DE000CF911F910F910895CF93DF93EC018881CC
:102DF0009981009711F00E945836198218821D821D
:102E00001C821B821A82DF91CF910895CF93DF93AA
:102E1000EC01FB0144815581608171810E948C1617
:102E2000811103C0CE010E94F416CE01DF91CF9133
:102E30000895EF92FF920F931F93CF93DF93EC01CE
:102E40007B018A01BA010E945A16811104C0CE0189
:102E50000E94F41607C01D830C83B70188819981F5
:102E60000E94BE37CE01DF91CF911F910F91FF904D
:102E7000EF900895CF93DF93EC016115710559F040
:102E8000FB0101900020E9F73197AF01461B570B7A
:102E90000E94191702C00E94F416CE01DF91CF9153
:102EA0000895CF93DF93EC01FB018617970761F03C
:102EB000608171816115710529F0448155810E94FD
:102EC000191702C00E94F416CE01DF91CF91089528
:102ED000FC01808191810C945836FC011182108292
:102EE00013821282158214826115710551F0FB0163
:102EF00001900020E9F73197AF01461B570B0C9466
:102F000019170895DB0114964D915C9115976D91F9
:102F10007C91DC01ED91FC910280F381E02D09941C
:102F20006115710579F0FB0101900020E9F73197F7
:102F3000AF01461B570BDC01ED91FC910280F38140
:102F4000E02D099480E090E008950C9490171F9272
:102F50000F920FB60F9211242F933F934F935F93CD
:102F60006F937F938F939F93AF93BF93EF93FF9351
:102F700085E695E00E94FE14FF91EF91BF91AF911D
:102F80009F918F917F916F915F914F913F912F9181
:102F90000F900FBE0F901F9018951F920F920FB6B3
:102FA0000F9211242F938F939F93EF93FF93E091B0
:102FB0007505F09176058081E0917B05F0917C05A7
:102FC00082FD12C0908180917E058F5F8F7320916A
:102FD0007F05821751F0E0917E05F0E0EB59FA4F42
:102FE000958F80937E0501C08081FF91EF919F9125
:102FF0008F912F910F900FBE0F901F9018951F92D9
:103000000F920FB60F9211242F933F934F935F931C
:103010006F937F938F939F93AF93BF93EF93FF93A0
:103020008091B900887F803609F49CC068F58832A9
:1030300009F45BC090F4803109F454C038F488235B
:1030400009F4F6C0883009F44DC0F6C0883109F49F
:103050004CC0803209F45DC0EFC0803409F468C010
:1030600048F4803309F455C0883309F0E5C08093F3
:103070003E05D8C0803509F44FC0883509F45DC0DD
:10308000883409F0D9C0D6C0883909F4C7C0A8F47B
:10309000883709F467C038F4883609F463C080378C
:1030A00009F460C0C9C0883809F4B8C0803909F48F
:1030B0005FC0803809F0C0C05BC0803B09F486C0A7
:1030C00038F4803A09F466C0883A09F47FC0B4C085
:1030D000803C09F4A7C0883C09F4A4C0883B09F4EB
:1030E0008AC0AAC080911B0510C090913D058091B7
:1030F0003C05981770F5E0913D0581E08E0F8093B7
:103100003D05F0E0E45EFA4F80818093BB0085ECE2
:1031100086C080933E058EC0E0913D0581E08E0F14
:1031200080933D058091BB00F0E0E45EFA4F808320
:1031300090913D0580913C056EC0E0913D0581E098
:103140008E0F80933D058091BB00F0E0E45EFA4F66
:10315000808380913F0581116DC081E080931A05C5
:1031600084EA61C083E08093400510921905CFCFB7
:1031700080911905803208F051C0E091190581E075
:103180008E0F809319058091BB00F0E0E750FB4F54
:103190008083BDCF85EC8093BC0010924005809168
:1031A0001905803230F4E0911905F0E0E750FB4F4B
:1031B00010826091190570E0E091B104F091B204C1
:1031C00089EF94E009951092190536C084E0809348
:1031D00040051092F8041092F704E091B304F091C6
:1031E000B40409958091F704811105C081E08093B2
:1031F000F7041092D704E091F80481E08E0F8093D9
:10320000F804F0E0E952FB4F80818093BB0090917D
:10321000F8048091F704981708F479CF85E8809333
:10322000BC000AC085EC8093BC001092400504C02D
:1032300010923E050E949915FF91EF91BF91AF91B9
:103240009F918F917F916F915F914F913F912F91BE
:103250000F900FBE0F901F901895FC01248131E054
:103260003093410520936305109242051092640546
:103270008385682B82E096E00E9426160C94101A33
:103280000F931F93CF938C01C62F0E942D196C2F83
:103290006460C8010E942D196C2F6B7FC8010E94C9
:1032A0002D1983EC90E00197F1F7CF911F910F91C9
:1032B00008950F931F93CF93DF938C01C62FD42FC4
:1032C000607F642B0E94401980E1C89FB0011124E7
:1032D0006D2BC801DF91CF911F910F910C94401974
:1032E00041E00E94591981E090E00895CF92DF9269
:1032F000EF92FF920F931F93CF93DF93EB017B012C
:1033000024E0E20EF11C8B016C01C61AD70AC6013B
:10331000800F911F0E944E32F80181938F01EE15AC
:10332000FF05A9F7CE01DF91CF911F910F91FF907B
:10333000EF90DF90CF9008950F931F93CF93DF937B
:1033400000D0CDB7DEB78B01FB0160819A83898302
:10335000CE0101960E949605C8010F900F90DF9153
:10336000CF911F910F910895AF92BF92CF92DF92AC
:10337000EF92FF920F931F93CF93DF9300D0CDB7BF
:10338000DEB78B016B0124E0C20ED11C7B015C0116
:10339000A61AB70AC5018E0D9F1DF70161917F0125
:1033A0009A838983CE0101960E949605EC14FD0450
:1033B00089F7C8010F900F90DF91CF911F910F9166
:1033C000FF90EF90DF90CF90BF90AF900895CF9394
:1033D000DF93EB010E944E328883CE01DF91CF91C3
:1033E000089580913801813029F480E096E9A0E0C9
:1033F000B0E00DC0823029F480E091EEA0E0B0E0B2
:1034000006C0833061F480E092ECA1E0B0E08093EC
:103410003E0190933F01A0934001B0934101089574
:1034200030916405313208F04BC080914005811124
:10343000FCCF9091630522E02093400521E020938A
:103440003F052FEF20933E0510923D0530933C053C
:10345000E3E4F5E0ACE1B5E020E0321721F0419182
:103460004D932F5FFACF10921B0520911B05990FEA
:10347000922B90931B0590911A05913061F4109254
:103480001A0590911B059093BB009091BC0093FD91
:10349000F8CF95EC01C095EE9093BC00909140055B
:1034A0009230E1F390913E059F3F79F080913E0587
:1034B000803241F080913E05803331F084E005C0D8
:1034C00081E003C082E001C083E0109242051092C7
:1034D0006405109241050895CF93DF93CDB7DEB711
:1034E00028970FB6F894DEBF0FBECDBF98E0E1E895
:1034F000F1E0DE01119601900D929A95E1F790911D
:10350000C206961710F46FEF690FFE013196E60FB1
:10351000F11DE60FF11D6081680F606840E08AEBE5
:1035200096E028960FB6F894DEBF0FBECDBFDF91B0
:10353000CF910C9459190F931F93CF93DF93CDB76D
:10354000DEB762970FB6F894DEBF0FBECDBF8C0119
:10355000FC011182108213821282158214824AE0C9
:10356000BE016F5F7F4F80E090E00E94AF30BE01F0
:103570006F5F7F4FC8010E943A1762960FB6F894AA
:10358000DEBF0FBECDBFDF91CF911F910F91089588
:10359000CF92DF92EF92FF926B017C01E091750573
:1035A000F091760582E08083C11481EED806E104B3
:1035B000F104B1F060E079E08DE390E0A7019601BD
:1035C0000E94DD33DA01C9010197A109B109B6955D
:1035D000A795979587959C01211580E13807B8F04C
:1035E000E0917505F0917605108260E874E88EE14F
:1035F00090E0A70196010E94DD33DA01C90101972D
:10360000A109B109B695A795979587959C01E09179
:103610007105F09172053083E0917305F0917405A6
:10362000208310927D05E0917905F0917A0586E07E
:103630008083E0917705F0917805808180618083B7
:10364000E0917705F0917805808188608083E09132
:103650007705F0917805808180688083E091770517
:10366000F091780580818F7D8083FF90EF90DF90CF
:10367000CF9008958F929F92AF92BF920F931F9316
:10368000CF93DF93CDB7DEB7A1970FB6F894DEBF27
:103690000FBECDBF19A2423008F44AE08E010F5D83
:1036A0001F4F842E912CA12CB12CA50194010E94B6
:1036B000DD33E62FB901CA0101501109EA3014F4D3
:1036C000E05D01C0E95CD801EC93232B242B252B72
:1036D00061F7B8018AEB96E00E949017A1960FB6A9
:1036E000F894DEBF0FBECDBFDF91CF911F910F9138
:1036F000BF90AF909F908F900895BC0180E090E0C4
:103700004AE00C943A1B41E0682F8AEB96E00E9455
:10371000591981E090E008950F931F93CF93DF93A1
:10372000CDB7DEB7A2970FB6F894DEBF0FBECDBF00
:103730008C01CB01BA01F80111821082138212822E
:10374000158214822AE0AE014F5F5F4F0E94BA30AB
:10375000BE016F5F7F4FC8010E943A17A2960FB655
:10376000F894DEBF0FBECDBFDF91CF911F910F91B7
:103770000895CF93DF93EC0141E050E065E172E002
:103780000E948C16811103C0CE010E94F416CE0156
:10379000DF91CF9108950F931F93CF93DF938B0108
:1037A00091E09093410590E6909363051092420555
:1037B00010926405682F82E096E00E942616E801C8
:1037C000085F1F4F699182E096E00E942616C0179D
:1037D000D107C1F7DF91CF911F910F910C94101A6F
:1037E0002F923F924F925F926F927F928F929F9211
:1037F000AF92BF92CF92DF92EF92FF920F931F93FF
:10380000CF93DF93CDB7DEB761970FB6F894DEBFE5
:103810000FBECDBF2D833E834F83588769877A873C
:103820001C011F870E876091B6067091B7068091C4
:10383000B8069091B90624E630E040E050E00E94DE
:103840008C342D87388B4B875C87762E672E582ECD
:10385000492E8091B0069091B106A091B206B09128
:10386000B3066C017D01FF0CCC08DC2C76019C01B9
:10387000AD016C2D7C2D8C2D9C2D0FE10E945735B8
:10388000A12C0AECB02EEAE9CE2EFBE3DF2EE12CD0
:10389000F12C00E010E00E94B934AD84B888CB84EC
:1038A000DC84E72CF62C052D142D0E9424340FE126
:1038B0000E94723549015A01D501C401BB0F880B22
:1038C000982FDC0189839A83AB83BC839401A50183
:1038D0006981762F862F962FAD84B888CB84DC84BF
:1038E000E72CF62C052D0E948E352983832E942EED
:1038F000598B688B7B878C879D872D813E814F817B
:10390000588569857A85C1012F3FA7E53A07A7E465
:103910004A07A8EF5A07ADE06A07710581059105CE
:10392000A9F0A0F0211534404B46544F6441710575
:1039300081059105B9F0B0F01D8294E09E83ABE65D
:10394000AF83B4EFB887E4E1E98709C01D82E8E5F9
:10395000EE83F7E4FF8328EF28878DE089871A86B6
:10396000212C312CA980B82CC92CD988E888FB845B
:103970000C851D852D813E814F81588569857A850D
:10398000C1010E94EA3429013A01FFE04F165104B7
:103990006104710418F4AFE0AA2E08C02BE54216AA
:1039A000510461047104D0F0FAE5AF2EB12CC12CA2
:1039B000D12CE12CF12C00E010E02981382D492D8B
:1039C000598968897B858C859D850E9424342D8347
:1039D0003E834F83588769877A871C01A980B82C5A
:1039E000C92CD988E888FB840C851D852D813E81F2
:1039F0004F81588569857A85C1010E94E834AA24DF
:103A0000AA94BB24BA94EFE0CE2ED12CE12CF12C59
:103A100000E010E00E942434A980B82CC92CD98879
:103A2000E888FB840C851D850E94EA34C901DA010F
:103A30000097A105B10529F4C12CD12C7601C394BE
:103A400006C0CC24CA94DC2C5FE0E52EF12CBC012E
:103A5000CD0127E0660F771F881F991F2A95D1F7A0
:103A600037E0440C551C661C771C3A95D1F7A2E050
:103A70005A1A61087108A70196010E94DD33862E4B
:103A8000372E982E420E531E641E751E84E190E060
:103A90000E94C0359A838983FC01D082C182862D21
:103AA0008370828353824482D701C6014CE0B6956D
:103AB000A795979587954A95D1F7807FC82EC90C11
:103AC000C582368287828E859F85892B19F4BF0136
:103AD0008AE107C0AE85BF85119729F469817A8193
:103AE00082E20E94CB1B89819A8161960FB6F8947D
:103AF000DEBF0FBECDBFDF91CF911F910F91FF9021
:103B0000EF90DF90CF90BF90AF909F908F907F907D
:103B10006F905F904F903F902F900C945836CF93BA
:103B2000C62F91E09093410590E690936305109223
:103B3000420510926405682F82E096E00E942616E6
:103B40006C2F82E096E00E942616CF910C94101AFA
:103B5000CF92DF92EF92FF920F931F93CF93DF9359
:103B60006C018B017A014617570720F4812F8A01D7
:103B7000E62EF82E66E372E0C6010E946D17C09132
:103B80007206D09173060C171D07E0F4EC16FD06C3
:103B900008F4E701E0916E06F0916F06EC0FFD1F4F
:103BA000F080108260916E0670916F06600F711F39
:103BB000C6010E943A1780916E0690916F06C80F59
:103BC000D91FF882C601DF91CF911F910F91FF900D
:103BD000EF90DF90CF9008953FB7F8948091CB0697
:103BE0009091CC06A091CD06B091CE0626B5A89BAB
:103BF00005C02F3F19F00196A11DB11D3FBFBA2F7F
:103C0000A92F982F8827820F911DA11DB11DBC01DE
:103C1000CD0142E0660F771F881F991F4A95D1F7A3
:103C20000895833081F028F4813099F08230A1F03A
:103C300008958730A9F08830B9F08430D1F48091AC
:103C400080008F7D03C0809180008F7780938000FB
:103C5000089584B58F7702C084B58F7D84BD0895A3
:103C60008091B0008F7703C08091B0008F7D8093EA
:103C7000B0000895CF93DF9390E0FC01E055FF4F33
:103C80002491FC01E456FF4F8491882361F190E078
:103C9000880F991FFC01E852FF4FC591D491FC0198
:103CA000E857FF4FA591B491611109C09FB7F894EF
:103CB0008881209582238883EC912E230BC062306B
:103CC00061F49FB7F8948881322F309583238883DD
:103CD000EC912E2B2C939FBF06C08FB7F894E881F0
:103CE0002E2B28838FBFDF91CF9108958E3008F05F
:103CF0008E508770806480937C0080917A0080640D
:103D000080937A0080917A0086FDFCCF80917800C4
:103D10002091790090E0922B08958F929F92AF921C
:103D2000BF92CF92DF92EF92FF926B017C010E94D3
:103D3000EC1D4B015C01C114D104E104F104F1F06C
:103D40000E94EC1DDC01CB0188199909AA09BB0965
:103D5000883E9340A105B10570F321E0C21AD10855
:103D6000E108F10888EE880E83E0981EA11CB11CC2
:103D7000C114D104E104F10419F7DDCFFF90EF90F5
:103D8000DF90CF90BF90AF909F908F9008952FB706
:103D9000F8946091C7067091C8068091C906909109
:103DA000CA062FBF08951F920F920FB60F921124CB
:103DB0002F933F938F939F93AF93BF938091C706A9
:103DC0009091C806A091C906B091CA063091C60666
:103DD00023E0230F2D3720F40196A11DB11D05C04E
:103DE00026E8230F0296A11DB11D2093C6068093DD
:103DF000C7069093C806A093C906B093CA068091DF
:103E0000CB069091CC06A091CD06B091CE0601963E
:103E1000A11DB11D8093CB069093CC06A093CD0637
:103E2000B093CE06BF91AF919F918F913F912F910B
:103E30000F900FBE0F901F901895CF93DF93CDB7C3
:103E4000DEB72C970FB6F894DEBF0FBECDBF7894C7
:103E500084B5826084BD84B5816084BD85B582608F
:103E600085BD85B5816085BD80916E008160809340
:103E70006E001092810080918100826080938100A9
:103E800080918100816080938100809180008160B9
:103E9000809380008091B10084608093B100809114
:103EA000B00081608093B00080917A00846080933C
:103EB0007A0080917A00826080937A0080917A0003
:103EC000816080937A0080917A00806880937A0084
:103ED0001092C1000E945A141092BF068091C4062D
:103EE000823018F098E09093BF068093C20662E398
:103EF00070E080E090E00E948D1E6091C5068AEB24
:103F000096E00E942D1968EE73E080E090E00E9438
:103F10008D1E60E38AEB96E00E9440190BE416E4E4
:103F2000C8010197F1F760E38AEB96E00E9440191F
:103F3000C8010197F1F760E38AEB96E00E9440190F
:103F400083E592E00197F1F760E28AEB96E00E9448
:103F500040196091BF06606240E08AEB96E00E94E3
:103F6000591984E08093C00640E06CE08AEB96E04B
:103F70000E9459190E949D1382E08093C10640E07F
:103F800066E08AEB96E00E94591940E062E08AEB15
:103F900096E00E9459198BE39FE10197F1F788E0C1
:103FA0008093C50660E08AEB96E00E942D196EE7CB
:103FB00074E080E090E00E94E719DC018C918E3D76
:103FC00009F031C78EE00E94761E843B91403CF0A0
:103FD0008EE00E94761E873192400CF424C768E37D
:103FE00071E088E290E00E94E719DC018C918093F7
:103FF000380168E371E088E290E00E94E719FC0173
:104000008081813031F460E076E980E090E00E94C8
:10401000C81A68E371E088E290E00E94E719DC01C9
:104020008C91823031F460E071EE80E090E00E948B
:10403000C81A68E371E088E290E00E94E719FC0189
:104040008081833031F460E072EC81E090E00E9486
:10405000C81A80913E0190913F01A0914001B0911A
:1040600041018115F6E99F07A105B10511F48FE023
:104070000EC0811521EE9207A105B10511F48AE069
:1040800006C08115924CA140B10519F488E08093D7
:10409000740461E084E00E943A1E60E085E00E94C2
:1040A0003A1E61E086E00E943A1E61E087E00E94CD
:1040B0003A1E61E088E00E943A1E61E089E00E94B9
:1040C0003A1E61E08AE00E943A1E61E08BE00E94A5
:1040D0003A1E61E08CE00E943A1E61E08DE00E9491
:1040E0003A1E60E080E10E943A1E60E081E10E9499
:1040F0003A1E62E080E10E943A1E62E085E00E9482
:104100003A1E62E081E10E943A1E8091680084605C
:104110008093680080916D008C6080936D0078942E
:104120006EE471E08CE390E00E94E719DC018C9171
:1041300080934E0166E471E08AE090E00E94761977
:10414000FC0180819181A281B3818093460190938B
:104150004701A0934801B093490162E471E084E112
:1041600090E00E947619FC0180819181A281B38147
:104170008093420190934301A0934401B093450181
:1041800064E776E08EE190E00E947619FC01808180
:104190009181A281B3818093740690937506A09358
:1041A0007606B09377066AE471E082E390E00E94BD
:1041B0007619FC0180819181A281B38180934A01AB
:1041C00090934B01A0934C01B0934D010E94B70313
:1041D00060917406709175068091760690917706CD
:1041E00024E630E040E050E00E947D342093570107
:1041F000309358014093590150935A0160935B01E9
:1042000070935C0180935D0190935E018091460103
:1042100090914701A0914801B09149018093B00667
:104220009093B106A093B206B093B306C09042013A
:10423000D0904301E0904401F09045010E945A144F
:1042400062E987EB0E948F1DC114D104E104F104DF
:1042500009F44EC08FE00E948C0C682F6F73F1E858
:10426000CF16F3ECDF06F9ECEF06F1E0FF0648F4B9
:10427000C092B606D092B706E092B806F092B906A0
:1042800034C0D701C6018158934CA94CB140803845
:10429000934CA94CB14070F4F694E794D794C7942A
:1042A000C092B606D092B706E092B806F092B90670
:1042B00060641BC0D701C60181509748A349B34031
:1042C00081159A45A246B24080F442E0F694E79404
:1042D000D794C7944A95D1F7C092B606D092B70644
:1042E000E092B806F092B90660688FE00E948F1DD8
:1042F00060E880E10E948F1D60E881E10E948F1DCF
:1043000060E882E10E948F1D6CE080E10E948F1DB9
:104310006CE081E10E948F1D6CE082E10E948F1DA4
:1043200060E281EB0E948F1D60E881EB0E948F1D8F
:1043300020915701309158014091590150915A01F3
:1043400060915B0170915C0180915D0190915E01D3
:1043500000E010E00E94F01BA0905701B0905801BF
:10436000C0905901D0905A01E0905B01F0905C013F
:1043700000915D0110915E0180914F01909150017B
:10438000A0915101B091520188529342A109B10903
:10439000BC01CD0122E0660F771F881F991F2A9567
:1043A000D1F724E630E040E050E00E947D34812CDB
:1043B000912C0E94E90D80E10E948C0C8C7F682F6B
:1043C000626080E10E948F1D60E371E081E00E94E5
:1043D000A81368E271E082E00E94A81360E271E035
:1043E00083E00E94A81368E171E084E00E94A813B2
:1043F00060E171E085E00E94A81368E071E086E06A
:104400000E94A81360E071E087E00E94A8130E9458
:104410009D1360E080E00E946C1A65EC71E08AEB0D
:1044200096E00E94A51761E080E00E946C1A66ED9C
:1044300071E08AEB96E00E94A51768EB7BE080E0D4
:1044400090E00E948D1E0E949D133CE0232E312C93
:1044500010927D040E94F11980917C04811102C0A8
:104460000E94B60880917B04811168C08091790414
:1044700090917A04892B09F061C080919C04882373
:10448000F1F08091810481111AC080917C04811126
:1044900016C080917D04882391F067EE71E085E677
:1044A00095E00E94A5176091740470E080E090E0B0
:1044B0000E948D1E81E0809381048093730480911B
:1044C0009C0481111BC0809181048823B9F08091E4
:1044D0007304882399F080917D04882379F06BEE32
:1044E00071E085E695E00E94A5176091740470E084
:1044F00080E090E00E948D1E1092810480917804EB
:10450000813081F480917C04811118C080917D04F8
:10451000882311F40C94062E61E084E00E942B1491
:104520000C94062E81110AC060E084E00E942B14D6
:1045300005C00530110514F00C943D2E80917804CF
:1045400081118FC08091790490917A04892B09F0B0
:1045500043C080917704882309F43EC085E695E046
:104560000E946D1560E172E085E695E00E94A51756
:104570006091740470E080E090E00E948D1E85E6FA
:1045800095E00E94E81418161906ECF466E372E050
:104590008EE696E00E943A1785E695E00E94E814C0
:1045A000181619066CF485E695E00E94C6140E9460
:1045B000ED1361E070E080E090E00E948D1EECCF92
:1045C00081E0809368048091680481110E94AF05A6
:1045D00080917804811145C08091790490917A048A
:1045E000892B09F087C080917704882309F482C061
:1045F00085E695E00E946D1567E172E085E695E03D
:104600000E94A5176AE070E080E090E00E948D1E95
:1046100085E695E00E94E81418161906ECF466E3A6
:1046200072E08EE696E00E943A1785E695E00E94D9
:10463000E814181619066CF485E695E00E94C61475
:104640000E94ED1361E070E080E090E00E948D1E1A
:10465000ECCF81E0809368048091680481110E940E
:10466000AF0580917804813009F044C080917604D0
:10467000813009F03FC08091790490917A04892BB0
:10468000C9F585E695E00E946D156DE172E085E65D
:1046900095E00E94A5176FE070E080E090E00E9436
:1046A0008D1E85E695E00E94E81418161906ECF4B4
:1046B00066E372E08EE696E00E943A1785E695E0A2
:1046C0000E94E814181619066CF485E695E00E941D
:1046D000C6140E94ED1361E070E080E090E00E945B
:1046E0008D1EECCF81E08093680480916804811175
:1046F0000E94AF0510917B041111D5C080917904FF
:1047000090917A04892B09F0CEC080917D04882392
:1047100009F4C9C080914F0190915001A0915101BD
:10472000B0915201813A9648A140B10584F480913C
:104730007C0481110CC080EA96E8A1E0B0E080938F
:104740004F0190935001A0935101B0935201809179
:104750004F0190915001A0915101B0915201803CC4
:104760009540A94DB14084F080917C0481110CC02A
:1047700080EC95E0A9EDB1E080934F01909350015A
:10478000A0935101B093520190916F0480917804ED
:104790009530B9F48130A9F480914F019091500186
:1047A000A0915101B0915201885F9A42A109B109CB
:1047B00080934F0190935001A0935101B093520107
:1047C00025C0811120C080916E04811106C08091A6
:1047D0006D0481110C94D22E09C0813009F063C0A0
:1047E00080916D04813011F00C94D82E80914F018E
:1047F00090915001A0915101B09152018852934281
:10480000A109B10948C0813009F04DC080916E0402
:10481000811149C080916D04813009F044C081E26A
:1048200092E00E94AF128823E1F040914F01509135
:1048300050016091510170915201809169049091F1
:104840006A04A0916B04B0916C04840F951FA61F9D
:10485000B71F80934F0190935001A0935101B093E3
:10486000520183E292E00E94AF128823E1F080912E
:104870004F0190915001A0915101B091520140918E
:10488000690450916A0460916B0470916C04841BFC
:10489000950BA60BB70B80934F0190935001A093FB
:1048A0005101B09352010E94E40380917704882360
:1048B00009F441C011113FC08091790490917A04AC
:1048C000892BC9F580917804811115C080917D04F0
:1048D000882389F08091980481110DC060E00E94C6
:1048E0006C1A65E272E08AEB96E00E94A51760E020
:1048F00084E00E942B14809178048130E1F480914F
:104900007D04882309F470C18091790490917A0420
:10491000892BB1F480919804811112C060E00E944B
:104920006C1A69E272E08AEB96E00E94A51761E0DA
:1049300084E00E942B1480917D04882309F454C1E3
:1049400080917B04811150C18091790490917A0407
:10495000892B09F049C180917804811145C10E94D9
:10496000C71E0E94C71EC0908C04D0908D04E0909A
:104970008E04F0908F04DC01CB018C199D09AE09E7
:10498000BF0984369105A105B10508F481C20E94D2
:10499000C71EDC01CB018C199D09AE09BF09843605
:1049A0009105A105B10570F00E94C71EDC01CB0185
:1049B0008C199D09AE09BF09883C9105A105B10577
:1049C00008F46FC20E94C71EDC01CB018C199D093F
:1049D000AE09BF09883C9105A105B10570F00E94A0
:1049E000C71EDC01CB018C199D09AE09BF098C32B1
:1049F0009140A105B10508F45DC20E94C71EDC010B
:104A0000CB018C199D09AE09BF098D329140A105DA
:104A1000B10508F4A8C000918A0410918B0480911C
:104A2000880490918904080F191F80918604909141
:104A30008704080F191F17FF02C00F5F1F4F15953E
:104A40000795109371040093700466E372E084E1AB
:104A500096E00E943A170C3811050CF034C2C801D8
:104A60004497B1010E94C933161617062CF0109214
:104A70008504109284045BC0709385046093840461
:104A80008091840490918504893091050CF18DE228
:104A900092E00E949E1261E08DE00E946C1A80916B
:104AA000820490918304181619060CF045C061E247
:104AB00072E08AEB96E00E94A517609182047091E3
:104AC0008304072E000C880B990B0E94741234C0CB
:104AD0008830910519F487E392E02BC08730910567
:104AE00019F487E492E025C08630910519F487E532
:104AF00092E01FC08530910519F487E692E019C055
:104B00008430910519F487E792E013C08330910552
:104B100019F487E892E00DC08230910519F487E915
:104B200092E007C0019719F487EA92E002C087EB90
:104B300092E00E949E1203C080E20E94831B61E00B
:104B400084E00E946C1A64E176E08AEB96E00E94B1
:104B500082170E94C71E60938C0470938D0480930B
:104B60008E0490938F048091780481113DC08091D0
:104B7000790490917A04892BB9F58091720481119E
:104B800009C061E00E946C1A69EC72E08AEB96E061
:104B90000E94A51780917204813051F461E080E099
:104BA0000E946C1A6EEC72E08AEB96E00E94A517E8
:104BB00080917204823051F461E080E00E946C1AAE
:104BC00063ED72E08AEB96E00E94A5178091720473
:104BD000833051F461E080E00E946C1A68ED72E06D
:104BE0008AEB96E00E94A5178EE00E94761E9093B5
:104BF0009304809392048438934034F080919B0412
:104C0000811102C010929A048EE00E94761E8C01DF
:104C100090939304809392040E94C71EDC01CB0101
:104C20000197A109B10985369105A105B10508F4DF
:104C3000E3C08EE00E94761E9C01235031090217CA
:104C4000130744F003968017910724F01093910402
:104C50000093900480919004909191048538A3E092
:104C60009A076CF080919D0410929B04811103C0FF
:104C700010929C04C1C081E080939C04BDC08F3120
:104C8000910534F520919B0430919D04211114C0AD
:104C9000311112C020917B0421111AC020917C0493
:104CA000211116C020917704222391F081E0809396
:104CB0009D0480939C0409C0332351F0211108C046
:104CC00010929D0410929C0481E080939B0494C0F8
:104CD0009C012F5231092A32310528F520919B047D
:104CE000211121C020919D0421111DC020919C04FF
:104CF000211119C08091390181508093390180912F
:104D0000790490917A04892B31F46DED72E085E697
:104D100095E00E94A51781E080939B046EE170E00E
:104D200080E090E049C09C012A55310924333105C7
:104D3000D0F420919B04211116C020919D042111D3
:104D400012C020919C0421110EC0809139018F5F07
:104D5000809339018091790490917A04892BD9F656
:104D600063EE72E0D4CF9C012F5831092D3231050A
:104D700030F520919B04211122C020919D04211126
:104D80001EC020919C0421111AC020917B04211186
:104D900016C08091790490917A04892B31F469EEE0
:104DA00072E085E695E00E94A51781E080939B0460
:104DB00068E270E080E090E00E948D1E1DC08D5B77
:104DC00091098B97C8F480919B04811115C0809143
:104DD0009D04811111C080919C0481110DC08091AE
:104DE0007B04811109C08091790490917A04892B08
:104DF000E1F66DEE72E0D5CF80E10E940214892BBE
:104E000069F480917C04811109C08091970481111B
:104E100005C080919E04882309F471C080919D048F
:104E200081116DC082C61A8219826EEDCE01019683
:104E30000E94960581E090E09A83898360E0CE012C
:104E400001960E94960566E471E08AE090E00E9477
:104E5000B41962E471E084E190E00E94B41964E75F
:104E600076E08EE190E00E94B41968E371E088E298
:104E700090E00E949C196AE471E082E390E00E9455
:104E8000B4196EE471E08CE390E00E949C19A7C80D
:104E9000809170049091710490938B0480938A04A4
:104EA00076CD8091700490917104909389048093E1
:104EB000880488CD80917004909171049093870448
:104EC000809386049ACD89E090E090938504809346
:104ED0008404B80166587109072E000C880B990BE1
:104EE0000E9431312FE832EC45EF5EE30E949031B1
:104EF0000E9489337093830460938204C1CD81E062
:104F000080939C048093730481E10E940214892B96
:104F100009F03DC0809173048823C9F160E080E00E
:104F20000E946C1A6DEB73E08AEB96E00E94A51765
:104F300080E2E82EF12C00E010E0809178060E94DB
:104F4000761E080F191FB1E0EB1AF108B1F7B8018E
:104F5000A5E075956795AA95E1F76F5F7140072EFB
:104F6000000C880B990B0E9431312FE135E847E1A5
:104F700052E40E94173342E00E94CF1261EF72E0C8
:104F80008AEB96E00E94A51780E20E94831B81E1D4
:104F90000E940214892B09F081C08091960481112E
:104FA0007DC080917304811179C0C2C564EF72E045
:104FB000CE0101960E946D17BE01695F7F4FCE0141
:104FC00001960E9406170E94B91BBC01CE010796EC
:104FD0000E945117CE0101960E946817BE01695FB9
:104FE0007F4F85E695E00E9482176091740470E01F
:104FF00080E090E00E948D1E67EF72E085E695E00C
:105000000E94A5176091740470E080E090E00E9417
:105010008D1EA0905701B0905801C0905901D090BA
:105020005A01E0905B01F0905C0100915D011091EC
:105030005E0180914A0190914B01A0914C01B09189
:105040004D0188529342A109B109BC01CD01F2E0A2
:10505000660F771F881F991FFA95D1F724E630E075
:1050600040E050E00E947D34812C912C0E94E90D9B
:1050700080914A0190914B01A0914C01B0914D015A
:1050800080934F0190935001A0935101B09352012E
:105090000E94E403CE0107960E94681781E10E94F6
:1050A0000214019721F48091960481119BC500910F
:1050B000790410917A040130110539F480919E042D
:1050C000811103C081E080939E0485E00E94021458
:1050D000019749F480919504811105C08091730472
:1050E000882309F482C585E00E940214892B21F4EB
:1050F00080919504811182C580919404811181C5AC
:1051000081E080937C048093970480917D048823C0
:10511000A9F180917B04811131C0012B79F5809137
:10512000780481112BC080919B04811127C080914C
:105130009A04811123C0809199048832F8F48091F7
:1051400098048823D9F060E080E00E946C1A6FEF29
:1051500072E08AEB96E00E94A51764E073E085E6B2
:1051600095E00E94A5176091740470E080E090E0E3
:105170000E948D1E10929804109299040091790457
:1051800010917A040115110509F062C080917B0429
:10519000811152C380917C04882309F445C0809119
:1051A0009D04811141C080919C0481113DC083E028
:1051B0000E948C0C682F6B7F83E00E948F1D2091D2
:1051C000770460914F01709150018091510190914D
:1051D0005201A0905701B0905801C0905901D09051
:1051E0005A01E0905B01F0905C0100915D0110912B
:1051F0005E01222321F0685D7C4D8F4F9F4F24E696
:1052000030E040E050E00E947D34E2E08E2E912CB0
:105210000E94E90D60E080E00E946C1A6AE073E091
:105220008AEB96E00E94A51780917C04811108C04A
:1052300083E00E948C0C682F646083E00E948F1DC5
:105240000091790410917A040115110509F4F4C252
:105250000E944D030130110509F0A8C06AE471E015
:1052600082E390E00E947619FC0180819181A28105
:10527000B38180934A0190934B01A0934C01B0936A
:105280004D0160E080E00E946C1A6EE073E08AEBF2
:1052900096E00E94A51780E20E94831B60914A015C
:1052A00070914B0180914C0190914D0120E432E4CA
:1052B0004FE050E00E94FF3369017A012A30310546
:1052C00018F480E20E94831BC6010E947D1B8EE2BF
:1052D0000E94831B60914A0170914B0180914C01A7
:1052E00090914D0120E432E44FE050E00E94FF3302
:1052F00028EE33E040E050E00E94FF3369017A017C
:1053000089012436310548F480E30E94831B0A306A
:10531000110518F480E30E94831BC6010E947D1BC7
:105320008EE20E94831B60914A0170914B01809133
:105330004C0190914D0128EE33E040E050E00E9496
:10534000FF336B017C018B016436710548F480E307
:105350000E94831B0A30110518F480E30E94831B0E
:10536000C6010E947D1B80E20E94831B61E080E0F9
:105370000E946C1A64E173E08AEB96E00E94A51724
:1053800060915301709154018091550190915601A3
:105390000E9474126BE173E08AEB96E00E94A517FD
:1053A00080E20E94831B80E20E94831B809179042B
:1053B00090917A04029709F0CEC06AE471E082E32A
:1053C00090E00E947619FC0180819181A281B381D5
:1053D00080934A0190934B01A0934C01B0934D01EF
:1053E00060E080E00E946C1A66E273E08AEB96E06F
:1053F0000E94A51780E20E94831B80914A01909130
:105400004B01A0914C01B0914D0188529342A109EA
:10541000B109BC01CD01B2E0660F771F881F991F4B
:10542000BA95D1F760939F047093A0048093A10470
:105430009093A20420E432E44FE050E00E94FF3356
:1054400069017A012A30310518F480E20E94831B39
:10545000C6010E947D1B8EE20E94831B60919F0407
:105460007091A0048091A1049091A20420E432E400
:105470004FE050E00E94FF3328EE33E040E050E080
:105480000E94FF3369017A0189012436310548F40D
:1054900080E30E94831B0A30110518F480E30E9408
:1054A000831BC6010E947D1B8EE20E94831B6091BC
:1054B0009F047091A0048091A1049091A20428EE11
:1054C00033E040E050E00E94FF336B017C018B0130
:1054D0006436710548F480E30E94831B0A3011058D
:1054E00018F480E30E94831BC6010E947D1B6CE2BE
:1054F00073E08AEB96E00E94A51761E080E00E94CD
:105500006C1A609146017091470180914801909119
:1055100049010E94741280E20E94831B61E087E0CF
:105520000E946C1A65E173E08AEB96E00E94A51771
:1055300060915301709154018091550190915601F1
:105540000E94741280E20E94831B80E20E94831BEF
:1055500080E20E94831B8091790490917A040397E2
:1055600039F560E080E00E946C1A60E373E08AEB3A
:1055700096E00E94A51761E080E00E946C1A62E448
:1055800072E08AEB96E00E94A51760917406709114
:10559000750680917606909177060E94741262E4F7
:1055A00072E08AEB96E00E94A51780E20E94831BBE
:1055B0008091790490917A04049739F560E080E055
:1055C0000E946C1A61E473E08AEB96E00E94A517D2
:1055D00061E080E00E946C1A62E472E08AEB96E07F
:1055E0000E94A5176091420170914301809144018E
:1055F000909145010E9474126CE273E08AEB96E090
:105600000E94A51780E20E94831B809179049091EB
:105610007A04059739F560E080E00E946C1A62E533
:1056200073E08AEB96E00E94A51761E080E00E949B
:105630006C1A63E673E08AEB96E00E94A51760910E
:105640003E0170913F0180914001909141010E9483
:10565000741262E472E08AEB96E00E94A51780E281
:105660000E94831B8091790490917A040697F1F54A
:105670006EE471E08CE390E00E94E719DC018C910C
:1056800080934E0160E080E00E946C1A6CE673E04B
:105690008AEB96E00E94A51780914E0161E0882375
:1056A000C1F080E00E946C1A60E472E08AEB96E040
:1056B0000E94A51760914E0170E080E090E04AE002
:1056C0000E943A1B6DE773E08AEB96E00E94A517F3
:1056D0000DC080E00E946C1A67E873E08AEB96E0E8
:1056E0000E94A5171092750410924E0180917904C2
:1056F00090917A0407970CF49FC010927A0410924C
:10570000790410929E0460E080E00E946C1A68E9BF
:1057100073E08AEB96E00E94A51761E080E00E94AA
:105720006C1A68EB72E08AEB96E00E94A517409134
:105730003A0150913B0160913C0170913D01CE01D5
:1057400007960E948C1B8B859C850B97A8F4CE0135
:1057500001960E949B1ABE01695F7F4FCE010196A0
:105760000E940617BC01CE0107960E945117CE0178
:1057700001960E946817E7CF64EF72E0CE010196B0
:105780000E946D17BE01695F7F4FCE0101960E9496
:1057900006170E94B91BBC01CE0107960E94511743
:1057A000CE0101960E946817BE01695F7F4F85E6B2
:1057B00095E00E9482176091740470E080E090E0B0
:1057C0000E948D1E69EA73E0CE0101960E946D175A
:1057D0006AE476E0CE0101960E9406170E94B91B8A
:1057E000BC018AE496E00E945117CE0101960E9406
:1057F00068176AE476E085E695E00E94821760917A
:10580000740470E080E090E00E948D1E66E372E018
:105810008AE496E00E943A1766E372E0CE010796AA
:105820000E943A1785E695E00E946D1510927B0460
:10583000CE0107960E94681780917C04882359F155
:1058400080917704811127C08091790490917A0426
:10585000892B09F50E944D030E941D0561E080E03F
:105860000E946C1A64E173E08AEB96E00E94A5172F
:1058700060915301709154018091550190915601AE
:105880000E9474126EEA73E08AEB96E00E94A517FC
:1058900080E20E94831B40904F0150905001609025
:1058A0005101709052018091A4049091A504A0919F
:1058B000A604B091A704481659066A067B06D9F1DA
:1058C00080917C04811137C080917704882399F1FD
:1058D0008091790490917A04892B69F5A090570101
:1058E000B0905801C0905901D0905A01E0905B01EE
:1058F000F0905C0100915D0110915E01C301B20165
:10590000A2E0660F771F881F991FAA95D1F724E69A
:1059100030E040E050E00E947D34812C912C0E94C8
:10592000E90D0E94E4034092A4045092A504609201
:10593000A6047092A7048091790490917A04892B2F
:10594000B9F180917704882399F1A0905701B09024
:105950005801C0905901D0905A01E0905B01F0903D
:105960005C0100915D0110915E01D301C20188527A
:105970009342A109B109BC01CD01F2E0660F771F86
:10598000881F991FFA95D1F724E630E040E050E0F7
:105990000E947D34812C912C0E94E90D0E94E40329
:1059A0004092A4045092A5046092A6047092A704A9
:1059B00020912A0630912B068091120690911306B1
:1059C0002817390729F580912606909127066091BE
:1059D0000E0670910F06009719F061157105A1F47C
:1059E0006115710549F0232B91F1FB01808190E055
:1059F0009195819591090AC0009749F1232B39F1BE
:105A0000DC018C9190E002C00E94B537892BF9F03F
:105A10008091760481111BC08091A304811117C06D
:105A200080917C04811113C080917704882379F0E0
:105A30006EE471E08CE390E00E94E719FC01808144
:105A400080934E010E94B70381E08093A30480916C
:105A5000A304882309F442C0809175048823F1F1DE
:105A600090914E019923D1F181508093750483E088
:105A70000E948C0C682F6D7F83E00E948F1DA09088
:105A80005701B0905801C0905901D0905A01E09050
:105A90005B01F0905C0100915D0110915E018091CD
:105AA0004F0190915001A0915101B0915201BC0160
:105AB000CD01685B7E488F4F9F4F24E630E040E089
:105AC00050E00E947D3488248394912C0E94E90D3B
:105AD00066E276E08EE096E00E94511780917504B0
:105AE000882321F080914E0181110AC083E00E9439
:105AF0008C0C682F626083E00E948F1D1092A304BB
:105B00008091A80481110DC080917704882349F009
:105B100066EB73E085E695E00E94A51781E080932F
:105B2000A8040E948F150C94282210929C04ECC9A2
:105B300081E0809396048091790490917A04019693
:105B400090937A0480937904019709F0A7CA809111
:105B50004F0190915001A0915101B0915201885D87
:105B60009C4DAF4FBF4F80933A0190933B01A09360
:105B70003C01B0933D0160E576E08AE496E00E9446
:105B800051176AE471E082E390E00E947619FC010B
:105B9000408151816281738140934A0150934B014E
:105BA00060934C0170934D01CE0107960E948C1BAF
:105BB0008B859C850B9708F0F9C9CE0101960E9450
:105BC0009B1ABE01695F7F4FCE0101960E940617A6
:105BD000BC01CE0107960E945117CE0101960E948A
:105BE0006817E6CF1092960462CA8091940491E0FF
:105BF0008927809394049093950475CA1092950414
:105C00007BCA10927C04109297047FCA80917D0415
:105C1000882311F40C949E2200917F04109180043B
:105C20000F5F1F4F1093800400937F0484E10E9454
:105C3000761EBC01990F880B990B0E9431316B01C4
:105C40007C0185E10E94761EBC01990F880B990B9F
:105C50000E9431312B013C019B01AC01C701B6010F
:105C60000E94BF3387FF02C00C94992261E080E05C
:105C70000E946C1A6FEE71E08FC010928004109237
:105C80007F04A3019201C701B6010E94AB324B0110
:105C90005C01A7019601C301B2010E94AA329B01D7
:105CA000AC01C501B4010E9417336B017C0120E0F7
:105CB00030E0A9010E94BF33181624F0F7FAF094DF
:105CC000F7F8F09420E030E040EA50E4C301B2017C
:105CD0000E94903120E030EC4FE754E40E941733EB
:105CE00029E23CE54FE85DE30E9417339B01AC01DC
:105CF0000E94903120E030E048E452E40E941733E3
:105D00002B013C0120E030E040E050E4C701B60147
:105D10000E94AB324B015C01A701960160E070E08C
:105D200080E89FE30E9417339B01AC01C501B401D9
:105D30000E94AB329B01AC0160E070E080E890E42F
:105D40000E941733A30192010E9490314B015C0124
:105D500061E080E00E946C1A62E072E08AEB96E0FB
:105D60000E94A51742E0C701B6010E94CF1261E070
:105D700088E00E946C1A67E072E08AEB96E00E946D
:105D8000A51761E08BE00E946C1A40E0C501B401E8
:105D90000E94CF126BE072E08AEB96E00E94A5179A
:105DA0000C949E22813011F00C9453240C94F62311
:105DB00081110C945324C0904F01D0905001E09079
:105DC0005101F090520198E2C91A93E2D90AE10810
:105DD000F108C0924F01D0925001E0925101F0922F
:105DE000520181E292E00E94AF12882311F40C94D8
:105DF00031248091690490916A04A0916B04B09160
:105E00006C04C80ED91EEA1EFB1EC0924F01D09230
:105E10005001E0925101F09252010C9431248EE035
:105E200096E00E94681784E196E00E9468178AE174
:105E300096E00E94681780E296E00E94681786E26A
:105E400096E00E9468178CE296E00E94681782E351
:105E500096E00E94681788E396E00E9468178EE338
:105E600096E00E94681784E496E00E9468178AE42E
:105E700096E00E94681780E596E00E94681786E524
:105E800096E00E9468178CE596E00E94681782E60B
:105E900096E00E94681788E696E00E9468178EE6F2
:105EA00096E00C946817AF92BF92CF92DF92EF9278
:105EB000FF920F931F93CF93DF93E5E6F5E01382F4
:105EC000128288EE93E0A0E0B0E084839583A683FD
:105ED000B7832DE831E03183208325EC30E035872E
:105EE000248724EC30E03787268720EC30E0318BA4
:105EF000208B21EC30E0338B228B22EC30E0358B91
:105F0000248B26EC30E0378B268B118E128E138E6D
:105F1000148EE2E0F6E01382128284839583A683D6
:105F2000B7838FE991E091838083EAEBF6E01382F7
:105F3000128281EB91E09183808387E2848380E108
:105F4000818782E082871386ECE7F6E098E090AFE5
:105F500091AF11AA12AA13AA11861286138614866B
:105F6000158616861786108A118A128A138A148A51
:105F7000158A168A178A108E118E128E138E148E21
:105F8000158E168E178E10A211A212A213A214A2A1
:105F900015A216A217A210A611A612A613A614A641
:105FA00015A616A617A610AA40E458E76DE771E0FB
:105FB00042AF53AF64AF75AFC9E7D6E0898383E0E2
:105FC0008A8360E082E00E943A1E60E08A810E943B
:105FD0003A1E61E089810E942B1461E08A810E944F
:105FE0002B1418828FE0809378062091570130910E
:105FF00058014091590150915A0160915B01709193
:106000005C0180915D0190915E01E4E6AE2EB12CC1
:10601000C12CD12CE12CF12C00E010E00E94EA34DC
:106020002093740630937506409376065093770656
:1060300066E372E08EE696E00E946D1766E372E01A
:1060400088E696E00E946D1766E372E082E696E0CD
:106050000E946D1766E372E08CE596E00E946D1772
:1060600066E372E086E596E00E946D1766E074E0F4
:1060700080E596E00E946D1766E372E08AE496E0A0
:106080000E946D1766E372E084E496E00E946D174B
:1060900066E372E08EE396E00E946D1766E372E0BD
:1060A00088E396E00E946D1766E372E082E396E073
:1060B0000E946D1766E372E08CE296E00E946D1715
:1060C00066E372E086E296E00E946D1766E372E096
:1060D00080E296E00E946D1766E372E08AE196E046
:1060E0000E946D1766E372E084E196E00E946D17EE
:1060F00066E372E08EE096E0DF91CF911F910F9101
:10610000FF90EF90DF90CF90BF90AF900C946D1701
:106110001F93FC0199278827BC01E8941191103244
:10612000E9F3193010F01E30C8F31B3251F01D3264
:1061300049F4689406C00E94C930610F711D811D29
:10614000911D119110531A30B0F33EF49095809543
:10615000709561957F4F8F4F9F4F1F910895BB277B
:106160004A3031F4992322F4BDE2909581959F4FF6
:106170000C940131BB272A3051F4992342F4BDE23B
:1061800090958095709561957F4F8F4F9F4F0C94A0
:10619000DF30592F482F372F262F660F771F881F84
:1061A000991F660F771F881F991F620F731F841F27
:1061B000951F660F771F881F991F0895BB27FA0147
:1061C000A62F6217710581059105330B30FB66F030
:1061D000AA27660F771F881F991FAA1FA21710F002
:1061E000A21B63953850A9F7A05DAA3308F0A95DFA
:1061F000A19336F7B111B1931082CA010C941A31F0
:10620000BB27FB015527AA27880F991FAA1FA41790
:1062100010F0A41B83955051B9F7A05DAA3308F084
:10622000A95DA193009779F7B111B1931192CB01B8
:106230000C941A31DC01FC01672F71917723E1F78F
:10624000329704C07C916D9370836291AE17BF0743
:10625000C8F308950E946C3108F481E00895E89431
:1062600009C097FB3EF490958095709561957F4F9E
:106270008F4F9F4F9923A9F0F92F96E9BB2793954C
:10628000F695879577956795B795F111F8CFFAF45C
:10629000BB0F11F460FF1BC06F5F7F4F8F4F9F4F8D
:1062A00016C0882311F096E911C0772321F09EE8EB
:1062B000872F762F05C0662371F096E8862F70E051
:1062C00060E02AF09A95660F771F881FDAF7880F2B
:1062D0009695879597F90895990F0008550FAA0B81
:1062E000E0E8FEEF16161706E807F907C0F01216E9
:1062F0001306E407F50798F0621B730B840B950BEC
:1063000039F40A2661F0232B242B252B21F4089540
:106310000A2609F4A140A6958FEF811D811D0895DD
:106320000E94A3310C9414320E94063238F00E946D
:106330000D3220F0952311F00C94FD310C940332B2
:1063400011240C9448320E94253270F3959FC1F3BA
:10635000950F50E0551F629FF001729FBB27F00D13
:10636000B11D639FAA27F00DB11DAA1F649F662768
:10637000B00DA11D661F829F2227B00DA11D621FB7
:10638000739FB00DA11D621F839FA00D611D221F71
:10639000749F3327A00D611D231F849F600D211D55
:1063A000822F762F6A2F11249F5750409AF0F1F0D8
:1063B00088234AF0EE0FFF1FBB1F661F771F881F41
:1063C00091505040A9F79E3F510580F00C94FD314B
:1063D0000C9448325F3FE4F3983ED4F3869577956A
:1063E0006795B795F795E7959F5FC1F7FE2B880FE7
:1063F000911D9695879597F9089597F99F6780E87D
:1064000070E060E008959FEF80EC089500240A9406
:106410001616170618060906089500240A9412167F
:106420001306140605060895092E0394000C11F4B2
:10643000882352F0BB0F40F4BF2B11F460FF04C05F
:106440006F5F7F4F8F4F9F4F089557FD9058440FB8
:10645000551F59F05F3F71F04795880F97FB991FC3
:1064600061F09F3F79F08795089512161306140680
:10647000551FF2CF4695F1DF08C01616170618060D
:10648000991FF1CF86957105610508940895E894E8
:10649000BB2766277727CB0197F90895F999FECF97
:1064A00092BD81BDF89A992780B50895262FF99954
:1064B000FECF1FBA92BD81BD20BD0FB6F894FA9AE7
:1064C000F99A0FBE019608952F923F924F925F92D4
:1064D0006F927F928F929F92AF92BF92CF92DF92F4
:1064E000EF92FF920F931F93CF93DF93CDB7DEB759
:1064F000CA1BDB0B0FB6F894DEBF0FBECDBF0994ED
:106500002A88398848885F846E847D848C849B8443
:10651000AA84B984C884DF80EE80FD800C811B8151
:10652000AA81B981CE0FD11D0FB6F894DEBF0FBE80
:10653000CDBFED010895A29FB001B39FC001A39FFD
:10654000700D811D1124911DB29F700D811D1124AC
:10655000911D08955058BB27AA270E94C2320C945F
:1065600014320E94063238F00E940D3220F039F4C5
:106570009F3F19F426F40C9403320EF4E095E7FBE8
:106580000C94FD31E92F0E94253258F3BA176207A7
:1065900073078407950720F079F4A6F50C94473229
:1065A0000EF4E0950B2EBA2FA02D0B01B90190012E
:1065B0000C01CA01A0011124FF27591B99F0593F72
:1065C00050F4503E68F11A16F040A22F232F342FBA
:1065D0004427585FF3CF469537952795A795F04008
:1065E0005395C9F77EF41F16BA0B620B730B840B1D
:1065F000BAF09150A1F0FF0FBB1F661F771F881FD5
:10660000C2F70EC0BA0F621F731F841F48F487952C
:1066100077956795B795F7959E3F08F0B0CF93951E
:10662000880F08F09927EE0F9795879508950E9497
:106630002B330C9414320E940D3258F00E94063213
:1066400040F029F45F3F29F00C94FD3151110C9476
:1066500048320C9403320E94253268F39923B1F337
:10666000552391F3951B550BBB27AA276217730778
:10667000840738F09F5F5F4F220F331F441FAA1F0C
:10668000A9F335D00E2E3AF0E0E832D091505040C8
:10669000E695001CCAF72BD0FE2F29D0660F771F76
:1066A000881FBB1F261737074807AB07B0E809F05C
:1066B000BB0B802DBF01FF2793585F4F3AF09E3FE1
:1066C000510578F00C94FD310C9448325F3FE4F3AF
:1066D000983ED4F3869577956795B795F7959F5F24
:1066E000C9F7880F911D9695879597F90895E1E070
:1066F000660F771F881FBB1F621773078407BA07CF
:1067000020F0621B730B840BBA0BEE1F88F7E09529
:1067100008950E9490336894B1110C944832089502
:106720000E942D3288F09F5798F0B92F9927B751C2
:10673000B0F0E1F0660F771F881F991F1AF0BA9525
:10674000C9F714C0B13091F00E944732B1E008950A
:106750000C944732672F782F8827B85F39F0B93FFC
:10676000CCF3869577956795B395D9F73EF49095D8
:106770008095709561957F4F8F4F9F4F08950E9430
:106780006C3108F48FEF08950E946C31880B990BDF
:10679000089597FB072E16F4009407D077FD09D0D3
:1067A0000E94AC3507FC05D03EF4909581959F4F33
:1067B0000895709561957F4F0895A1E21A2EAA1B46
:1067C000BB1BFD010DC0AA1FBB1FEE1FFF1FA217A1
:1067D000B307E407F50720F0A21BB30BE40BF50B9E
:1067E000661F771F881F991F1A9469F76095709527
:1067F000809590959B01AC01BD01CF010895052EB8
:1068000097FB1EF400940E94163457FD07D00E9497
:10681000DD3307FC03D04EF40C94163450954095AC
:10682000309521953F4F4F4F5F4F0895909580953C
:10683000709561957F4F8F4F9F4F0895EE0FFF1F0B
:106840000590F491E02D0994DF93CF931F930F935C
:106850009A9DF02D219FF00D8B9DF00D8A9DE02DCE
:10686000F10D039FF00D029FE00DF11D4E9DE00D17
:10687000F11D5E9DF00D4F9DF00D7F936F93BF92C4
:10688000AF925F934F93D5010E949B328B01AC0175
:10689000D7010E949B32EB01E80FF91FD6010E943D
:1068A00074342F913F91D6010E949B32C60FD71F9F
:1068B000E81FF91FAF91BF910E9474342F913F914F
:1068C0000E949B32C60FD71FE81FF91FD6010E94F6
:1068D0009B32E60FF71F9801BE01CF0111240F91E3
:1068E0001F91CF91DF9108950E949B32460F571F51
:1068F000C81FD91F08F43196089597FB57FF0C94D1
:106900008D349F938F930E948D346E1B7F0BAF91BC
:10691000BF918A0B9B0B0895E894DF93CF93FC0102
:10692000DB010E949B327F936F93E9019A01AC01D6
:10693000BF93AF933F932F93DF010E949B3226F4C6
:106940006C1B7D0B820B930B9E01EB01FC010E94E3
:106950007434AF91BF912F913F910E947434BE0166
:10696000CF01F9012F913F91CF91DF910895689464
:1069700001C0E894F92FF12B12F00C94EB34A0E055
:10698000B0E0E5ECF4E30C946A32092E059422F4AD
:106990000E944735112392F4F0E80F26FFEFE094B0
:1069A000F09400951095B094C094D094A194BF0A2F
:1069B000CF0ADF0AEF0AFF0A0F0B1F0B0E94F63403
:1069C00007FC0E944735CDB7DEB7ECE00C94863269
:1069D000689401C0E8948F929F92CF93DF930E94B6
:1069E000F634DF91CF919F908F9008958824992459
:1069F000F401E401B0E49F93AA279A158B049C0448
:106A0000ED05FE05CF05D007A10798F4AD2FDC2FCB
:106A1000CF2FFE2FE92D982C892E982F872F762F98
:106A2000652F542F432F322F2227B85031F7BF91B3
:106A300027C01B2EBF91BB27220F331F441F551F9A
:106A4000661F771F881F991F881C991CEE1FFF1F48
:106A5000CC1FDD1FAA1FBB1F8A149B04EC05FD057C
:106A6000CE05DF05A007B10748F08A189B08EC099E
:106A7000FD09CE09DF09A00BB10B21601A94E1F6E4
:106A80002EF49401AF01BE01CD01000C0895609574
:106A900070958095909530954095509521953F4FF4
:106AA0004F4F5F4F6F4F7F4F8F4F9F4F08950F9303
:106AB000083090F0982F872F762F652F542F432F73
:106AC000322F22270850F4CF220F331F441F551FA7
:106AD000661F771F881F991F0A95B2F70F910895B7
:106AE00097FB10F8169400080F93083098F00850A0
:106AF000232F342F452F562F672F782F892F902D36
:106B0000F4CF059497958795779567955795479511
:106B1000379527950A95AAF70F9108952A0D3B1DE1
:106B20004C1D5D1D6E1D7F1D801F911F08952A1530
:106B30003B054C055D056E057F05800791070895AF
:106B40000024A7FD00942A17300540055005600574
:106B50007005800590050895AA1BBB1B51E107C075
:106B6000AA1FBB1FA617B70710F0A61BB70B881FDD
:106B7000991F5A95A9F780959095BC01CD0108956C
:106B80000F931F93CF93DF938230910510F482E02F
:106B900090E0E091D106F091D20620E030E0A0E054
:106BA000B0E0309719F1408151810281138148177B
:106BB0005907C8F08417950769F4109731F01296B9
:106BC0000C93129713961C9327C00093D106109331
:106BD000D20622C02115310519F04217530718F4C7
:106BE0009A01BD01EF01DF01F801DBCF211531056D
:106BF000F9F0281B390B2430310580F48A819B8100
:106C00006115710521F0FB019383828304C0909389
:106C1000D2068093D106FE01329644C0FE01E20FF7
:106C2000F31F8193919322503109398328833AC00D
:106C30002091CF063091D006232B41F420916101A1
:106C4000309162013093D0062093CF0620915F01EE
:106C5000309160012115310541F42DB73EB74091C7
:106C6000630150916401241B350BE091CF06F09134
:106C7000D006E217F307A0F42E1B3F0B28173907A5
:106C800078F0AC014E5F5F4F2417350748F04E0F88
:106C90005F1F5093D0064093CF068193919302C01B
:106CA000E0E0F0E0CF01DF91CF911F910F910895C7
:106CB000CF93DF93009709F481C0FC0132971382D0
:106CC0001282A091D106B091D206109781F4208152
:106CD0003181820F931F2091CF063091D006281763
:106CE000390751F5F093D006E093CF0667C0ED0168
:106CF00020E030E0CE17DF0740F44A815B819E013F
:106D000041155105F1F0EA01F5CFD383C2834081EB
:106D10005181840F951FC817D90759F4888199812B
:106D2000840F951F0296918380838A819B81938330
:106D300082832115310529F4F093D206E093D10620
:106D40003DC0E901FB83EA8349915991C40FD51FE6
:106D5000EC17FD0761F480819181840F951F0296E5
:106D6000E90199838883828193819B838A83E0E010
:106D7000F0E012968D919C911397009719F0FD0108
:106D8000DC01F7CF8D919C9111979D012E5F3F4FB4
:106D9000820F931F2091CF063091D0062817390714
:106DA00069F4309729F41092D2061092D10602C0ED
:106DB00013821282B093D006A093CF06DF91CF91B9
:106DC0000895A0E0B0E0E7EEF6E30C946832EC0141
:106DD000009721F4CB010E94C035B4C0FC01E60F3E
:106DE000F71F9C0122503109E217F30708F4A8C0ED
:106DF000D9010D911C91119706171707B0F00530B6
:106E0000110508F49BC0C80104978617970708F47A
:106E100095C002501109061B170B019311936D9336
:106E20007C93CF010E94583689C05B01A01AB10A39
:106E30004C01800E911EA091D106B091D206612C1A
:106E4000712CE12CF12C109709F446C08D919C9186
:106E50001197A815B905B1F56C0142E0C40ED11C1B
:106E6000CA14DB0478F14C018A189B08640142E0E3
:106E7000C40ED11C1296BC9012971396AC91B5E03B
:106E8000CB16D10440F0B282A38391828082D901D3
:106E90006D937C9309C00E5F1F4F800F911FF90106
:106EA00091838083EB2DFA2FE114F10431F0D701A7
:106EB0001396FC93EE93129741C0F093D206E093A1
:106EC000D1063CC06816790608F43C017D01129693
:106ED0000D90BC91A02DB7CF8091CF069091D00698
:106EE00088169906E1F466167706C8F480915F016A
:106EF00090916001009741F48DB79EB74091630176
:106F000050916401841B950BE817F907C8F4F093BE
:106F1000D006E093CF06F901718360830FC0CB01E7
:106F20000E94C0357C01009759F0A801BE010E9463
:106F3000AC37CE010E945836C70104C0CE0102C052
:106F400080E090E0CDB7DEB7EEE00C94843281E0D3
:106F500090E0F8940C94D337FB01DC0102C001905F
:106F60000D9241505040D8F70895FB01DC018D91FE
:106F7000019080190110D9F3990B0895FB01DC01F0
:106F800001900D920020E1F70895FB01DC014150D2
:106F9000504030F08D910190801919F40020B9F71C
:106FA000881B990B089510E0C2E7D0E004C0FE01F1
:106FB0000E941E342196C337D107C9F7F894FFCF3A
:106FC0001F1115111D1D111F1F1115111515111F51
:106FD0001F111D1D1D1D1D1F1F1117111515111F1F
:106FE0001F1117111D1D111F1F1515111D1D1D1F0F
:106FF0001F111D111D1D111F0207D0B1370000E127
:107000000000C0FC9B01400D0300A03B4C0005505C
:1070100073370040420F00002E5976110000000027
:1070200000D30680000002040003000110030200E8
:107030000003020100060004000605002006050406
:107040000000004000140054000000000020158DD6
:1070500014B7146D15E814C614DA140000000026E5
:1070600016F9155516CD15F115DD15CE15000000D4
:107070000070198D1455168C140000000058168DE0
:107080001455168C145344522053696E74657A203B
:107090005554334D4B00536F66742E204D69636B0E
:1070A000795F76302E340054583B0052583B0053E1
:1070B0005752202020202020503D305720202020D3
:1070C00020005357523D0020503D00572020200003
:1070D0005A5A534D303B005A5A50413B0046423BAE
:1070E000002B002D005258200054582000FFFFFFB5
:1070F000FFFFFFFFFF0700FFFFFFFFFFFFFF06206F
:1071000020202020202000FFFFFFFFFFFF05202080
:1071100020202020202000FFFFFFFFFF0420202050
:1071200020202020202000FFFFFFFF032020202020
:1071300020202020202000FFFFFF022020202020F0
:1071400020202020202000FFFF01202020202020C0
:1071500020202020202000FFFF2020202020202091
:1071600020202020202000FF202020202020202060
:10717000202020202020002020202020202020202F
:107180002020202020202020004F666620004C6F09
:107190007720004D6564200048696768005A5A539B
:1071A000443B005A5A53553B0042553B0042443B36
:1071B000002041004641005A5A4D4430323B004CB9
:1071C0006F6164005A5A51523B0056666F00467216
:1071D00043616C002053746570200020487A2020A1
:1071E00020202020200043725265660020487A004B
:1071F00020436F72722E504C4C5F464958454420D4
:1072000000436F7272465245512E205155415254DF
:107210005A00434F4D20504F52542052532D323379
:107220003220002020426175643A200020457261BE
:107230007365207369646562616E64200020205369
:10724000656320202020002020202020204F66661B
:1072500020202020202020002020524553544F522F
:107260004520467265712020005A5A4D440020483E
:107270007A20202020005A5A5352303B00416D7032
:1072800065722E203D200055503B00444E3B00319E
:1072900036300038300034300033300032300031C6
:1072A00037003135003132003130004F0045525245
:1072B0004F5220535445503E32354B487A003F00E0
:1072C0004946003030003032003034003035003074
:1072D00036003039003033003037005A5A534D30C1
:1072E000005A5A50410046420049463B00202020A7
:1072F000444953434F4E4E45435420202000202004
:107300002020506F776572534452202020202000A7
:1073100055415254002042617564006E616E0069EF
:087320006E66006F7666000046
:00000001FF
